:020000040000FA
:3C000000FFFF627515FFFFFFFFFFFFFFFFFFFFFFFFFFFFFFFFFFFFFFFFFFFFFFFFFFFFFFFFFFFFFFFFFFFFFFFFFFFFFFFFFFFFFFFFFFFFFFFFFFFFFFFFFFFFFF11
:3C003C00000000000000000000000000000000000000000000000000000000000000000000000000000000000000000000000000000000000000000000001EFE6C
:3C007800000000000000000000000000000000000000000000000000000000000000000000000000000000000000000000000000000000000000000000001EFE30
:3C00B4000000000000000000000004800000000000000000000000000000000000000000000004000400000000000000000000000080040000000000000092FE70
:3C00F000000004800480048004800480048004800480048004800480048004800480048004800480048004800480048004800480048004800480048000001EFECC
:3C012C00000004800480048004800480048004800480048004800480048004800480048004800480048004800480048004800480048004800480048000001EFE8F
:3C016800000004000480000000000480000000000480040004800080040004000000000000000400048004000480008004000480008004800400048000001AFEFF
:3C01A4000000008000000480048004800480048000000080000004000080008004800480048004800400008000000400008000000480040000800000000096FED3
:3C01E0000000008000000480048004800480048000000080000004000080008004800480048004800400008000000400008000000480040000800000000096FE97
:3C021C00000000000000000000000000000000000000000000000000000000000000000000000000000000000000000000000000000000000000000000001EFE8A
:3C025800000000000000000000000000000000000000000000000000000000000000000000000000000000000000000000000000000000000000000000001EFE4E
:3C029400000000000000000000000000000000000000000000000000000000000000000000000000000000000000000000000000000000000000000000001EFE12
:3C02D000020000000000000000000000000000000000000000000000000000000000000000000000000000000000000000000000000000000000000000002FFFC2
:3C030C00020000000000000000000000000000000000000000000000000000000000000000000000000000000000000000000000000000000000000000002FFF85
:3C034800020000000000000000000000000000000000000000000000000000000000000000000000000000000000000000000000000000000000000000002FFF49
:3C038400000000000000000000000000000000000000000000000000000000000000000000000000000000000000000000000000000000000000000000001EFE21
:3C03C000000000000000000000000000000000000000000000000000000000000000000000000000000000000000000000000000000000000000000000001EFEE5
:3C03FC00000000000000000000000000000000000000000000000000000000000000000000000000000000000000000000000000000000000000000000001EFEA9
:3C043800000000000000000000000000000000000000000000000000000000000000000000000000000000000000000000000000000000000000000000001EFE6C
:3C047400000000000000000000000000000000000000000000000000000000000000000000000000000000000000000000000000000000000000000000001EFE30
:3C04B000020000000000000000000000000000000000000000000000000000000000000000000000000000000000000000000000000000000000000000002FFFE0
:3C04EC00020000000000000000000000000000000000000000000000000000000000000000000000000000000000000000000000000000000000000000002FFFA4
:3C052800000000000000000000000000000000000000000000000000000000000000000000000000000000000000000000000000000000000000000000001EFE7B
:3C056400020000000000000000000000000000000000000000000000000000000000000000000000000000000000000000000000000000000000000000002FFF2B
:3C05A000020000000000000000000000000000000000000000000000000000000000000000000000000000000000000000000000000000000000000000002FFFEF
:3C05DC00000000000000000000000000000000000000000000000000000000000000000000000000000000000000000000000000000000000000000000001EFEC7
:3C061800000000000000000000000000000000000000000000000000000000000000000000000000000000000000000000000000000000000000000000001EFE8A
:3C065400000000000000000000000000000000000000000000000000000000000000000000000000000000000000000000000000000000000000000000001EFE4E
:3C069000020000000000000000000000000000000000000000000000000000000000000000000000000000000000000000000000000000000000000000002FFFFE
:3C06CC00020000000000000000000000000000000000000000000000000000000000000000000000000000000000000000000000000000000000000000002FFFC2
:3C070800020000000000000000000000000000000000000000000000000000000000000000000000000000000000000000000000000000000000000000002FFF85
:3C074400000000000000000000000000000000000000000000000000000000000000000000000000000000000000000000000000000000000000000000001EFE5D
:3C078000000000000000000000000000000000000000000000000000000000000000000000000000000000000000000000000000000000000000000000001EFE21
:3C07BC00000000000000000000000000000000000000000000000000000000000000000000000000000000000000000000000000000000000000000000001EFEE5
:3C07F800000000000000000000000000000000000000000000000000000000000000000000000000000000000000000000000000000000000000000000001EFEA9
:3C083400000000000000000000000000000000000000000000000000000000000000000000000000000000000000000000000000000000000000000000001EFE6C
:3C087000020000000000000000000000000000000000000000000000000000000000000000000000000000000000000000000000000000000000000000002FFF1C
:3C08AC00020000000000000000000000000000000000000000000000000000000000000000000000000000000000000000000000000000000000000000002FFFE0
:3C08E800020000000000000000000000000000000000000000000000000000000000000000000000000000000000000000000000000000000000000000002FFFA4
:3C092400000000000000000000000000000000000000000000000000000000000000000000000000000000000000000000000000000000000000000000001EFE7B
:3C096000000000000000000000000000000000000000000000000000000000000000000000000000000000000000000000000000000000000000000000001EFE3F
:3C099C00000000000000000000000000000000000000000000000000000000000000000000000000000000000000000000000000000000000000000000001EFE03
:3C09D800000000000000000000000000000000000000000000000000000000000000000000000000000000000000000000000000000000000000000000001EFEC7
:3C0A1400000000000000000000000000000000000000000000000000000000000000000000000000000000000000000000000000000000000000000000001EFE8A
:3C0A5000020000000000000000000000000000000000000000000000000000000000000000000000000000000000000000000000000000000000000000002FFF3A
:3C0A8C00020000000000000000000000000000000000000000000000000000000000000000000000000000000000000000000000000000000000000000002FFFFE
:3C0AC800020000000000000000000000000000000000000000000000000000000000000000000000000000000000000000000000000000000000000000002FFFC2
:3C0B0400000000000000000000000000000000000000000000000000000000000000000000000000000000000000000000000000000000000000000000001EFE99
:3C0B4000000000000000000000000000000000000000000000000000000000000000000000000000000000000000000000000000000000000000000000001EFE5D
:3C0B7C00000000000000000000000000000000000000000000000000000000000000000000000000000000000000000000000000000000000000000000001EFE21
:3C0BB800000000000000000000000000000000000000000000000000000000000000000000000000000000000000000000000000000000000000000000001EFEE5
:3C0BF400000000000000000000000000000000000000000000000000000000000000000000000000000000000000000000000000000000000000000000001EFEA9
:3C0C3000020000000000000000000000000000000000000000000000000000000000000000000000000000000000000000000000000000000000000000002FFF58
:3C0C6C00020000000000000000000000000000000000000000000000000000000000000000000000000000000000000000000000000000000000000000002FFF1C
:3C0CA800020000000000000000000000000000000000000000000000000000000000000000000000000000000000000000000000000000000000000000003EFED2
:3C0CE400000000000000000000000000000000000000000000000000000000000000000000000000000000000000000000000000000000000000000000000FFFC6
:3C0D2000000000000000000000000000000000000000000000000000000000000000000000000000000000000000000000000000000000000000000000000FFF89
:3C0D5C00000000000000000000000000000000000000000000000000000000000000000000000000000000000000000000000000000000000000000000001EFE3F
:3C0D9800000000000000000000000000000000000000000000000000000000000000000000000000000000000000000000000000000000000000000000001EFE03
:3C0DD400000000000000000000000000000000000000000000000000000000000000000000000000000000000000000000000000000000000000000000001EFEC7
:3C0E1000020000000000000000000000000000000000000000000000000000000000000000000000000000000000000000000000000000000000000000002FFF76
:3C0E4C00020000000000000000000000000000000000000000000000000000000000000000000000000000000000000000000000000000000000000000002FFF3A
:3C0E8800000000000000000000000000000000000000000000000000000000000000000000000000000000000000000000000000000000000000000000001EFE12
:3C0EC400020000000000000000000000000000000000000000000000000000000000000000000000000000000000000000000000000000000000000000002FFFC2
:3C0F0000020000000000000000000000000000000000000000000000000000000000000000000000000000000000000000000000000000000000000000002FFF85
:3C0F3C00000000000000000000000000000000000000000000000000000000000000000000000000000000000000000000000000000000000000000000001EFE5D
:3C0F7800000000000000000000000000000000000000000000000000000000000000000000000000000000000000000000000000000000000000000000001EFE21
:3C0FB400000000000000000000000000000000000000000000000000000000000000000000000000000000000000000000000000000000000000000000001EFEE5
:3C0FF000020000000000000000000000000000000000000000000000000000000000000000000000000000000000000000000000000000000000000000002FFF95
:3C102C00020000000000000000000000000000000000000000000000000000000000000000000000000000000000000000000000000000000000000000002FFF58
:3C106800000000000000000000000000000000000000000000000000000000000000000000000000000000000000000000000000000000000000000000001EFE30
:3C10A400020000000000000000000000000000000000000000000000000000000000000000000000000000000000000000000000000000000000000000002FFFE0
:3C10E000020000000000000000000000000000000000000000000000000000000000000000000000000000000000000000000000000000000000000000002FFFA4
:3C111C00000000000000000000000000000000000000000000000000000000000000000000000000000000000000000000000000000000000000000000001EFE7B
:3C115800000000000000000000000000000000000000000000000000000000000000000000000000000000000000000000000000000000000000000000001EFE3F
:3C119400000000000000000000000000000000000000000000000000000000000000000000000000000000000000000000000000000000000000000000001EFE03
:3C11D000020000000000000000000000000000000000000000000000000000000000000000000000000000000000000000000000000000000000000000002FFFB3
:3C120C00020000000000000000000000000000000000000000000000000000000000000000000000000000000000000000000000000000000000000000002FFF76
:3C124800000000000000000000000000000000000000000000000000000000000000000000000000000000000000000000000000000000000000000000001EFE4E
:3C128400020000000000000000000000000000000000000000000000000000000000000000000000000000000000000000000000000000000000000000002FFFFE
:3C12C000020000000000000000000000000000000000000000000000000000000000000000000000000000000000000000000000000000000000000000002FFFC2
:3C12FC00000000000000000000000000000000000000000000000000000000000000000000000000000000000000000000000000000000000000000000001EFE9A
:3C133800000000000000000000000000000000000000000000000000000000000000000000000000000000000000000000000000000000000000000000001EFE5D
:3C137400000000000000000000000000000000000000000000000000000000000000000000000000000000000000000000000000000000000000000000001EFE21
:3C13B000020000000000000000000000000000000000000000000000000000000000000000000000000000000000000000000000000000000000000000002FFFD1
:3C13EC00020000000000000000000000000000000000000000000000000000000000000000000000000000000000000000000000000000000000000000002FFF95
:3C142800008000800080008000800080008000800080008000800080008000800080008000800080008000800080008000800080008000800080008000009EFEEC
:3C146400020000000000000000000000000000000000000000000000000000000000000000000000000000000000000000000000000000000000000000002FFF1C
:3C14A000020000000000000000000000000000000000000000000000000000000000000000000000000000000000000000000000000000000000000000002FFFE0
:3C14DC00000000000000000000000000000000000000000000000000000000000000000000000000000000000000000000000000000000000000000000001EFEB8
:3C151800000000000000000000000000000000000000000000000000000000000000000000000000000000000000000000000000000000000000000000001EFE7B
:3C155400000000000000000000000000000000000000000000000000000000000000000000000000000000000000000000000000000000000000000000001EFE3F
:3C159000000000000000000000000000000000000000000000000000000000000000000000000000000000000000000000000000000000000000000000001EFE03
:3C15CC00000000000000000000000000000000000000000000000000000000000000000000000000000000000000000000000000000000000000000000001EFEC7
:3C160800000000000000000000000000000000000000000000000000000000000000000000000000000000000000000000000000000000000000000000001EFE8A
:3C164400000000000000000000000000000000000000000000000000000000000000000000000000000000000000000000000000000000000000000000001EFE4E
:3C168000000000000000000000000000000000000000000000000000000000000000000000000000000000000000000000000000000000000000000000001EFE12
:3C16BC00000000000000000000000000000000000000000000000000000000000000000000000000000000000000000000000000000000000000000000001EFED6
:3C16F800000000000000000000000000000000000000000000000000000000000000000000000000000000000000000000000000000000000000000000001EFE9A
:3C173400000000000000000000000000000000000000000000000000000000000000000000000000000000000000000000000000000000000000000000001EFE5D
:3C177000000000000000000000000000000000000000000000000000000000000000000000000000000000000000000000000000000000000000000000001EFE21
:3C17AC00000000000000000000000000000000000000000000000000000000000000000000000000000000000000000000000000000000000000000000001EFEE5
:3C17E800000000000000000000000000000000000000000000000000000000000000000000000000000000000000000000000000000000000000000000001EFEA9
:3C182400000000000000000000000000000000000000000000000000000000000000000000000000000000000000000000000000000000000000000000001EFE6C
:3C186000000000000000000000000000000000000000000000000000000000000000000000000000000000000000000000000000000000000000000000001EFE30
:3C189C00000000000000000000000000000000000000000000000000000000000000000000000000000000000000000000000000000000000000000000001EFEF4
:3C18D800000000000000000000000000000000000000000000000000000000000000000000000000000000000000000000000000000000000000000000001EFEB8
:3C191400000000000000000000000000000000000000000000000000000000000000000000000000000000000000000000000000000000000000000000001EFE7B
:3C195000000000000000000000000000000000000000000000000000000000000000000000000000000000000000000000000000000000000000000000001EFE3F
:3C198C00000000000000000000000000000000000000000000000000000000000000000000000000000000000000000000000000000000000000000000001EFE03
:3C19C800000000000000000000000000000000000000000000000000000000000000000000000000000000000000000000000000000000000000000000001EFEC7
:3C1A0400000000000000000000000000000000000000000000000000000000000000000000000000000000000000000000000000000000000000000000001EFE8A
:3C1A4000000000000000000000000000000000000000000000000000000000000000000000000000000000000000000000000000000000000000000000001EFE4E
:3C1A7C00000000000000000000000000000000000000000000000000000000000000000000000000000000000000000000000000000000000000000000001EFE12
:3C1AB800000000000000000000000000000000000000000000000000000000000000000000000000000000000000000000000000000000000000000000001EFED6
:3C1AF400000000000000000000000000000000000000000000000000000000000000000000000000000000000000000000000000000000000000000000001EFE9A
:3C1B3000000000000000000000000000000000000000000000000000000000000000000000000000000000000000000000000000000000000000000000001EFE5D
:3C1B6C00000000000000000000000000000000000000000000000000000000000000000000000000000000000000000000000000000000000000000000001EFE21
:3C1BA800000000000000000000000000000000000000000000000000000000000000000000000000000000000000000000000000000000000000000000001EFEE5
:3C1BE400000000000000000000000000000000000000000000000000000000000000000000000000000000000000000000000000000000000000000000001EFEA9
:3C1C2000000000000000000000000000000000000000000000000000000000000000000000000000000000000000000000000000000000000000000000001EFE6C
:3C1C5C00000000000000000000000000000000000000000000000000000000000000000000000000000000000000000000000000000000000000000000001EFE30
:3C1C9800000000000000000000000000000000000000000000000000000000000000000000000000000000000000000000000000000000000000000000001EFEF4
:3C1CD400000000000000000000000000000000000000000000000000000000000000000000000000000000000000000000000000000000000000000000001EFEB8
:3C1D1000000000000000000000000000000000000000000000000000000000000000000000000000000000000000000000000000000000000000000000001EFE7B
:3C1D4C00000000000000000000000000000000000000000000000000000000000000000000000000000000000000000000000000000000000000000000000FFF4D
:3C1D8800000000000000000000000000000000000000000000000000000000000000000000000000000000000000000000000000000000000000000000001EFE03
:3C1DC400000000000000000000000000000000000000000000000000000000000000000000000000000000000000000000000000000000000000000000001EFEC7
:3C1E0000020000000000000000000000000000000000000000000000000000000000000000000000000000000000000000000000000000000000000000003EFE68
:3C1E3C00020000000000000000000000000000000000000000000000000000000000000000000000000000000000000000000000000000000000000000002FFF3A
:3C1E7800000000000000000000000000000000000000000000000000000000000000000000000000000000000000000000000000000000000000000000000FFF20
:3C1EB400020000000000000000000000000000000000000000000000000000000000000000000000000000000000000000000000000000000000000000003EFEB4
:3C1EF000020000000000000000000000000000000000000000000000000000000000000000000000000000000000000000000000000000000000000000003EFE78
:3C1F2C00020000000000000000000000000000000000000000000000000000000000000000000000000000000000000000000000000000000000000000003EFE3B
:3C1F6800000000000000000000000000000000000000000000000000000000000000000000000000000000000000000000000000000000000000000000001EFE21
:3C1FA400000000000000000000000000000000000000000000000000000000000000000000000000000000000000000000000000000000000000000000001EFEE5
:3C1FE000020000000000000000000000000000000000000000000000000000000000000000000000000000000000000000000000000000000000000000002FFF95
:3C201C00020000000000000000000000000000000000000000000000000000000000000000000000000000000000000000000000000000000000000000002FFF58
:3C205800020000000000000000000000000000000000000000000000000000000000000000000000000000000000000000000000000000000000000000002FFF1C
:3C209400020000000000000000000000000000000000000000000000000000000000000000000000000000000000000000000000000000000000000000003EFED2
:3C20D000020000000000000000000000000000000000000000000000000000000000000000000000000000000000000000000000000000000000000000003EFE96
:3C210C00000000000000000000000000000000000000000000000000000000000000000000000000000000000000000000000000000000000000000000001EFE7B
:3C214800000000000000000000000000000000000000000000000000000000000000000000000000000000000000000000000000000000000000000000001EFE3F
:3C218400000000000000000000000000000000000000000000000000000000000000000000000000000000000000000000000000000000000000000000001EFE03
:3C21C000020000000000000000000000000000000000000000000000000000000000000000000000000000000000000000000000000000000000000000002FFFB3
:3C21FC00020000000000000000000000000000000000000000000000000000000000000000000000000000000000000000000000000000000000000000002FFF77
:3C223800000000000000000000000000000000000000000000000000000000000000000000000000000000000000000000000000000000000000000000001EFE4E
:3C227400020000000000000000000000000000000000000000000000000000000000000000000000000000000000000000000000000000000000000000002FFFFE
:3C22B000020000000000000000000000000000000000000000000000000000000000000000000000000000000000000000000000000000000000000000002FFFC2
:3C22EC00020000000000000000000000000000000000000000000000000000000000000000000000000000000000000000000000000000000000000000003EFE78
:3C232800000000000000000000000000000000000000000000000000000000000000000000000000000000000000000000000000000000000000000000001EFE5D
:3C236400000000000000000000000000000000000000000000000000000000000000000000000000000000000000000000000000000000000000000000001EFE21
:3C23A000020000000000000000000000000000000000000000000000000000000000000000000000000000000000000000000000000000000000000000002FFFD1
:3C23DC00020000000000000000000000000000000000000000000000000000000000000000000000000000000000000000000000000000000000000000002FFF95
:3C241800020000000000000000000000000000000000000000000000000000000000000000000000000000000000000000000000000000000000000000003EFE4A
:3C245400020000000000000000000000000000000000000000000000000000000000000000000000000000000000000000000000000000000000000000002FFF1C
:3C249000020000000000000000000000000000000000000000000000000000000000000000000000000000000000000000000000000000000000000000002FFFE0
:3C24CC00000000000000000000000000000000000000000000000000000000000000000000000000000000000000000000000000000000000000000000000FFFC6
:3C250800000000000000000000000000000000000000000000000000000000000000000000000000000000000000000000000000000000000000000000001EFE7B
:3C254400000000000000000000000000000000000000000000000000000000000000000000000000000000000000000000000000000000000000000000001EFE3F
:3C258000020000000000000000000000000000000000000000000000000000000000000000000000000000000000000000000000000000000000000000003EFEE1
:3C25BC00020000000000000000000000000000000000000000000000000000000000000000000000000000000000000000000000000000000000000000002FFFB3
:3C25F800000000000000000000000000000000000000000000000000000000000000000000000000000000000000000000000000000000000000000000000FFF99
:3C263400020000000000000000000000000000000000000000000000000000000000000000000000000000000000000000000000000000000000000000003EFE2C
:3C267000020000000000000000000000000000000000000000000000000000000000000000000000000000000000000000000000000000000000000000003EFEF0
:3C26AC00000000000000000000000000000000000000000000000000000000000000000000000000000000000000000000000000000000000000000000001EFED6
:3C26E800000000000000000000000000000000000000000000000000000000000000000000000000000000000000000000000000000000000000000000001EFE9A
:3C272400000000000000000000000000000000000000000000000000000000000000000000000000000000000000000000000000000000000000000000001EFE5D
:3C276000020000000000000000000000000000000000000000000000000000000000000000000000000000000000000000000000000000000000000000002FFF0D
:3C279C00020000000000000000000000000000000000000000000000000000000000000000000000000000000000000000000000000000000000000000002FFFD1
:3C27D800000000000000000000000000000000000000000000000000000000000000000000000000000000000000000000000000000000000000000000001EFEA9
:3C281400020000000000000000000000000000000000000000000000000000000000000000000000000000000000000000000000000000000000000000002FFF58
:3C285000020000000000000000000000000000000000000000000000000000000000000000000000000000000000000000000000000000000000000000002FFF1C
:3C288C00000000000000000000000000000000000000000000000000000000000000000000000000000000000000000000000000000000000000000000000FFF02
:3C28C800000000000000000000000000000000000000000000000000000000000000000000000000000000000000000000000000000000000000000000001EFEB8
:3C290400000000000000000000000000000000000000000000000000000000000000000000000000000000000000000000000000000000000000000000001EFE7B
:3C294000020000000000000000000000000000000000000000000000000000000000000000000000000000000000000000000000000000000000000000003EFE1D
:3C297C00020000000000000000000000000000000000000000000000000000000000000000000000000000000000000000000000000000000000000000002FFFEF
:3C29B800000000000000000000000000000000000000000000000000000000000000000000000000000000000000000000000000000000000000000000000FFFD5
:3C29F400020000000000000000000000000000000000000000000000000000000000000000000000000000000000000000000000000000000000000000003EFE69
:3C2A3000020000000000000000000000000000000000000000000000000000000000000000000000000000000000000000000000000000000000000000003EFE2C
:3C2A6C00000000000000000000000000000000000000000000000000000000000000000000000000000000000000000000000000000000000000000000000FFF20
:3C2AA800000000000000000000000000000000000000000000000000000000000000000000000000000000000000000000000000000000000000000000001EFED6
:3C2AE400000000000000000000000000000000000000000000000000000000000000000000000000000000000000000000000000000000000000000000001EFE9A
:3C2B2000020000000000000000000000000000000000000000000000000000000000000000000000000000000000000000000000000000000000000000003EFE3B
:3C2B5C00020000000000000000000000000000000000000000000000000000000000000000000000000000000000000000000000000000000000000000002FFF0D
:3C2B9800000000000000000000000000000000000000000000000000000000000000000000000000000000000000000000000000000000000000000000000FFFF3
:3C2BD400020000000000000000000000000000000000000000000000000000000000000000000000000000000000000000000000000000000000000000003EFE87
:3C2C1000020000000000000000000000000000000000000000000000000000000000000000000000000000000000000000000000000000000000000000003EFE4A
:3C2C4C00000000000000000000000000000000000000000000000000000000000000000000000000000000000000000000000000000000000000000000001EFE30
:3C2C8800000000000000000000000000000000000000000000000000000000000000000000000000000000000000000000000000000000000000000000001EFEF4
:3C2CC400000000000000000000000000000000000000000000000000000000000000000000000000000000000000000000000000000000000000000000001EFEB8
:3C2D0000020000000000000000000000000000000000000000000000000000000000000000000000000000000000000000000000000000000000000000002FFF67
:3C2D3C00020000000000000000000000000000000000000000000000000000000000000000000000000000000000000000000000000000000000000000002FFF2B
:3C2D7800020000000000000000000000000000000000000000000000000000000000000000000000000000000000000000000000000000000000000000003EFEE1
:3C2DB400000000000000000000000000000000000000000000000000000000000000000000000000000000000000000000000000000000000000000000000FFFD5
:3C2DF000000000000000000000000000000000000000000000000000000000000000000000000000000000000000000000000000000000000000000000000FFF99
:3C2E2C00000000000000000000000000000000000000000000000000000000000000000000000000000000000000000000000000000000000000000000000FFF5C
:3C2E6800000000000000000000000000000000000000000000000000000000000000000000000000000000000000000000000000000000000000000000001EFE12
:3C2EA400000000000000000000000000000000000000000000000000000000000000000000000000000000000000000000000000000000000000000000001EFED6
:3C2EE000020000000000000000000000000000000000000000000000000000000000000000000000000000000000000000000000000000000000000000003EFE78
:3C2F1C00020000000000000000000000000000000000000000000000000000000000000000000000000000000000000000000000000000000000000000002FFF49
:3C2F5800008000800080008000800080008000800080008000800080008000800080008000800080008000800080008000800080008000800080008000008FFFAF
:3C2F9400020000000000000000000000000000000000000000000000000000000000000000000000000000000000000000000000000000000000000000003EFEC3
:3C2FD000020000000000000000000000000000000000000000000000000000000000000000000000000000000000000000000000000000000000000000003EFE87
:3C300C00000000000000000000000000000000000000000000000000000000000000000000000000000000000000000000000000000000000000000000001EFE6C
:3C304800000000000000000000000000000000000000000000000000000000000000000000000000000000000000000000000000000000000000000000001EFE30
:3C308400000000000000000000000000000000000000000000000000000000000000000000000000000000000000000000000000000000000000000000001EFEF4
:3C30C000000000000000000000000000000000000000000000000000000000000000000000000000000000000000000000000000000000000000000000001EFEB8
:3C30FC00000000000000000000000000000000000000000000000000000000000000000000000000000000000000000000000000000000000000000000001EFE7C
:3C313800000000000000000000000000000000000000000000000000000000000000000000000000000000000000000000000000000000000000000000001EFE3F
:3C317400000000000000000000000000000000000000000000000000000000000000000000000000000000000000000000000000000000000000000000001EFE03
:3C31B000000000000000000000000000000000000000000000000000000000000000000000000000000000000000000000000000000000000000000000001EFEC7
:3C31EC00000000000000000000000000000000000000000000000000000000000000000000000000000000000000000000000000000000000000000000001EFE8B
:3C322800000000000000000000000000000000000000000000000000000000000000000000000000000000000000000000000000000000000000000000001EFE4E
:3C326400000000000000000000000000000000000000000000000000000000000000000000000000000000000000000000000000000000000000000000001EFE12
:3C32A000000000000000000000000000000000000000000000000000000000000000000000000000000000000000000000000000000000000000000000001EFED6
:3C32DC00000000000000000000000000000000000000000000000000000000000000000000000000000000000000000000000000000000000000000000001EFE9A
:3C331800000000000000000000000000000000000000000000000000000000000000000000000000000000000000000000000000000000000000000000001EFE5D
:3C335400000000000000000000000000000000000000000000000000000000000000000000000000000000000000000000000000000000000000000000001EFE21
:3C339000000000000000000000000000000000000000000000000000000000000000000000000000000000000000000000000000000000000000000000001EFEE5
:3C33CC00000000000000000000000000000000000000000000000000000000000000000000000000000000000000000000000000000000000000000000001EFEA9
:3C340800000000000000000000000000000000000000000000000000000000000000000000000000000000000000000000000000000000000000000000001EFE6C
:3C344400000000000000000000000000000000000000000000000000000000000000000000000000000000000000000000000000000000000000000000001EFE30
:3C348000000000000000000000000000000000000000000000000000000000000000000000000000000000000000000000000000000000000000000000001EFEF4
:3C34BC00000000000000000000000000000000000000000000000000000000000000000000000000000000000000000000000000000000000000000000001EFEB8
:3C34F800000000000000000000000000000000000000000000000000000000000000000000000000000000000000000000000000000000000000000000001EFE7C
:3C353400000000000000000000000000000000000000000000000000000000000000000000000000000000000000000000000000000000000000000000001EFE3F
:3C357000000000000000000000000000000000000000000000000000000000000000000000000000000000000000000000000000000000000000000000001EFE03
:3C35AC00000000000000000000000000000000000000000000000000000000000000000000000000000000000000000000000000000000000000000000001EFEC7
:3C35E800000000000000000000000000000000000000000000000000000000000000000000000000000000000000000000000000000000000000000000001EFE8B
:3C362400000000000000000000000000000000000000000000000000000000000000000000000000000000000000000000000000000000000000000000001EFE4E
:3C366000000000000000000000000000000000000000000000000000000000000000000000000000000000000000000000000000000000000000000000001EFE12
:3C369C00000000000000000000000000000000000000000000000000000000000000000000000000000000000000000000000000000000000000000000001EFED6
:3C36D800000000000000000000000000000000000000000000000000000000000000000000000000000000000000000000000000000000000000000000001EFE9A
:3C371400000000000000000000000000000000000000000000000000000000000000000000000000000000000000000000000000000000000000000000001EFE5D
:3C375000000000000000000000000000000000000000000000000000000000000000000000000000000000000000000000000000000000000000000000001EFE21
:3C378C00000000000000000000000000000000000000000000000000000000000000000000000000000000000000000000000000000000000000000000001EFEE5
:3C37C800000000000000000000000000000000000000000000000000000000000000000000000000000000000000000000000000000000000000000000001EFEA9
:3C380400000000000000000000000000000000000000000000000000000000000000000000000000000000000000000000000000000000000000000000001EFE6C
:3C384000000000000000000000000000000000000000000000000000000000000000000000000000000000000000000000000000000000000000000000001EFE30
:3C387C00000000000000000000000000000000000000000000000000000000000000000000000000000000000000000000000000000000000000000000001EFEF4
:3C38B800000000000000000000000000000000000000000000000000000000000000000000000000000000000000000000000000000000000000000000001EFEB8
:3C38F400000000000000000000000000000000000000000000000000000000000000000000000000000000000000000000000000000000000000000000001EFE7C
:3C393000020000000000000000000000000000000000000000000000000000000000000000000000000000000000000000000000000000000000000000002FFF2B
:3C396C00020000000000000000000000000000000000000000000000000000000000000000000000000000000000000000000000000000000000000000002FFFEF
:3C39A800000000000000000000000000000000000000000000000000000000000000000000000000000000000000000000000000000000000000000000001EFEC7
:3C39E400020000000000000000000000000000000000000000000000000000000000000000000000000000000000000000000000000000000000000000002FFF77
:3C3A2000020000000000000000000000000000000000000000000000000000000000000000000000000000000000000000000000000000000000000000002FFF3A
:3C3A5C00000000000000000000000000000000000000000000000000000000000000000000000000000000000000000000000000000000000000000000001EFE12
:3C3A9800000000000000000000000000000000000000000000000000000000000000000000000000000000000000000000000000000000000000000000001EFED6
:3C3AD400000000000000000000000000000000000000000000000000000000000000000000000000000000000000000000000000000000000000000000001EFE9A
:3C3B1000020000000000000000000000000000000000000000000000000000000000000000000000000000000000000000000000000000000000000000002FFF49
:3C3B4C00020000000000000000000000000000000000000000000000000000000000000000000000000000000000000000000000000000000000000000002FFF0D
:3C3B8800020000000000000000000000000000000000000000000000000000000000000000000000000000000000000000000000000000000000000000003EFEC3
:3C3BC400000000000000000000000000000000000000000000000000000000000000000000000000000000000000000000000000000000000000000000000FFFB7
:3C3C0000000000000000000000000000000000000000000000000000000000000000000000000000000000000000000000000000000000000000000000000FFF7A
:3C3C3C00000000000000000000000000000000000000000000000000000000000000000000000000000000000000000000000000000000000000000000000FFF3E
:3C3C7800000000000000000000000000000000000000000000000000000000000000000000000000000000000000000000000000000000000000000000001EFEF4
:3C3CB400000000000000000000000000000000000000000000000000000000000000000000000000000000000000000000000000000000000000000000001EFEB8
:3C3CF000020000000000000000000000000000000000000000000000000000000000000000000000000000000000000000000000000000000000000000002FFF68
:3C3D2C00020000000000000000000000000000000000000000000000000000000000000000000000000000000000000000000000000000000000000000002FFF2B
:3C3D6800020000000000000000000000000000000000000000000000000000000000000000000000000000000000000000000000000000000000000000002FFFEF
:3C3DA400000000000000000000000000000000000000000000000000000000000000000000000000000000000000000000000000000000000000000000000FFFD5
:3C3DE000000000000000000000000000000000000000000000000000000000000000000000000000000000000000000000000000000000000000000000000FFF99
:3C3E1C00000000000000000000000000000000000000000000000000000000000000000000000000000000000000000000000000000000000000000000000FFF5C
:3C3E5800000000000000000000000000000000000000000000000000000000000000000000000000000000000000000000000000000000000000000000001EFE12
:3C3E9400000000000000000000000000000000000000000000000000000000000000000000000000000000000000000000000000000000000000000000001EFED6
:3C3ED000020000000000000000000000000000000000000000000000000000000000000000000000000000000000000000000000000000000000000000002FFF86
:3C3F0C00020000000000000000000000000000000000000000000000000000000000000000000000000000000000000000000000000000000000000000002FFF49
:3C3F4800020000000000000000000000000000000000000000000000000000000000000000000000000000000000000000000000000000000000000000002FFF0D
:3C3F8400000000000000000000000000000000000000000000000000000000000000000000000000000000000000000000000000000000000000000000000FFFF3
:3C3FC000000000000000000000000000000000000000000000000000000000000000000000000000000000000000000000000000000000000000000000000FFFB7
:3C3FFC00000000000000000000000000000000000000000000000000000000000000000000000000000000000000000000000000000000000000000000000FFF7B
:3C403800000000000000000000000000000000000000000000000000000000000000000000000000000000000000000000000000000000000000000000001EFE30
:3C407400000000000000000000000000000000000000000000000000000000000000000000000000000000000000000000000000000000000000000000001EFEF4
:3C40B000020000000000000000000000000000000000000000000000000000000000000000000000000000000000000000000000000000000000000000002FFFA4
:3C40EC00020000000000000000000000000000000000000000000000000000000000000000000000000000000000000000000000000000000000000000002FFF68
:3C412800020000000000000000000000000000000000000000000000000000000000000000000000000000000000000000000000000000000000000000002FFF2B
:3C416400000000000000000000000000000000000000000000000000000000000000000000000000000000000000000000000000000000000000000000000FFF11
:3C41A000000000000000000000000000000000000000000000000000000000000000000000000000000000000000000000000000000000000000000000000FFFD5
:3C41DC00000000000000000000000000000000000000000000000000000000000000000000000000000000000000000000000000000000000000000000000FFF99
:3C421800000000000000000000000000000000000000000000000000000000000000000000000000000000000000000000000000000000000000000000001EFE4E
:3C425400000000000000000000000000000000000000000000000000000000000000000000000000000000000000000000000000000000000000000000001EFE12
:3C429000020000000000000000000000000000000000000000000000000000000000000000000000000000000000000000000000000000000000000000002FFFC2
:3C42CC00020000000000000000000000000000000000000000000000000000000000000000000000000000000000000000000000000000000000000000002FFF86
:3C430800020000000000000000000000000000000000000000000000000000000000000000000000000000000000000000000000000000000000000000002FFF49
:3C434400000000000000000000000000000000000000000000000000000000000000000000000000000000000000000000000000000000000000000000000FFF2F
:3C438000000000000000000000000000000000000000000000000000000000000000000000000000000000000000000000000000000000000000000000000FFFF3
:3C43BC00000000000000000000000000000000000000000000000000000000000000000000000000000000000000000000000000000000000000000000001EFEA9
:3C43F800000000000000000000000000000000000000000000000000000000000000000000000000000000000000000000000000000000000000000000001EFE6D
:3C443400000000000000000000000000000000000000000000000000000000000000000000000000000000000000000000000000000000000000000000001EFE30
:3C447000020000000000000000000000000000000000000000000000000000000000000000000000000000000000000000000000000000000000000000002FFFE0
:3C44AC00020000000000000000000000000000000000000000000000000000000000000000000000000000000000000000000000000000000000000000002FFFA4
:3C44E800000000000000000000000000000000000000000000000000000000000000000000000000000000000000000000000000000000000000000000001EFE7C
:3C452400020000000000000000000000000000000000000000000000000000000000000000000000000000000000000000000000000000000000000000002FFF2B
:3C456000020000000000000000000000000000000000000000000000000000000000000000000000000000000000000000000000000000000000000000002FFFEF
:3C459C00000000000000000000000000000000000000000000000000000000000000000000000000000000000000000000000000000000000000000000000FFFD5
:3C45D800000000000000000000000000000000000000000000000000000000000000000000000000000000000000000000000000000000000000000000001EFE8B
:3C461400000000000000000000000000000000000000000000000000000000000000000000000000000000000000000000000000000000000000000000001EFE4E
:3C465000020000000000000000000000000000000000000000000000000000000000000000000000000000000000000000000000000000000000000000003EFEF0
:3C468C00020000000000000000000000000000000000000000000000000000000000000000000000000000000000000000000000000000000000000000002FFFC2
:3C46C800020000000000000000000000000000000000000000000000000000000000000000000000000000000000000000000000000000000000000000002FFF86
:3C470400000000000000000000000000000000000000000000000000000000000000000000000000000000000000000000000000000000000000000000001EFE5D
:3C474000000000000000000000000000000000000000000000000000000000000000000000000000000000000000000000000000000000000000000000001EFE21
:3C477C00000000000000000000000000000000000000000000000000000000000000000000000000000000000000000000000000000000000000000000000FFFF3
:3C47B800000000000000000000000000000000000000000000000000000000000000000000000000000000000000000000000000000000000000000000001EFEA9
:3C47F400000000000000000000000000000000000000000000000000000000000000000000000000000000000000000000000000000000000000000000001EFE6D
:3C483000020000000000000000000000000000000000000000000000000000000000000000000000000000000000000000000000000000000000000000003EFE0E
:3C486C00020000000000000000000000000000000000000000000000000000000000000000000000000000000000000000000000000000000000000000002FFFE0
:3C48A800020000000000000000000000000000000000000000000000000000000000000000000000000000000000000000000000000000000000000000002FFFA4
:3C48E400000000000000000000000000000000000000000000000000000000000000000000000000000000000000000000000000000000000000000000000FFF8A
:3C492000000000000000000000000000000000000000000000000000000000000000000000000000000000000000000000000000000000000000000000000FFF4D
:3C495C00020000000000000000000000000000000000000000000000000000000000000000000000000000000000000000000000000000000000000000002FFFEF
:3C499800000000000000000000000000000000000000000000000000000000000000000000000000000000000000000000000000000000000000000000001EFEC7
:3C49D400000000000000000000000000000000000000000000000000000000000000000000000000000000000000000000000000000000000000000000001EFE8B
:3C4A1000000000000000000000000000000000000000000000000000000000000000000000000000000000000000000000000000000000000000000000001EFE4E
:3C4A4C00000000000000000000000000000000000000000000000000000000000000000000000000000000000000000000000000000000000000000000001EFE12
:3C4A8800008000800080008000800080008000800080008000800080008000800080008000800080008000800080008000800080008000800080008000009EFE56
:3C4AC400000000000000000000000000000000000000000000000000000000000000000000000000000000000000000000000000000000000000000000001EFE9A
:3C4B0000000000000000000000000000000000000000000000000000000000000000000000000000000000000000000000000000000000000000000000001EFE5D
:3C4B3C00000000000000000000000000000000000000000000000000000000000000000000000000000000000000000000000000000000000000000000001EFE21
:3C4B7800000000000000000000000000000000000000000000000000000000000000000000000000000000000000000000000000000000000000000000001EFEE5
:3C4BB400000000000000000000000000000000000000000000000000000000000000000000000000000000000000000000000000000000000000000000001EFEA9
:3C4BF000000000000000000000000000000000000000000000000000000000000000000000000000000000000000000000000000000000000000000000001EFE6D
:3C4C2C00000000000000000000000000000000000000000000000000000000000000000000000000000000000000000000000000000000000000000000001EFE30
:3C4C6800000000000000000000000000000000000000000000000000000000000000000000000000000000000000000000000000000000000000000000001EFEF4
:3C4CA400000000000000000000000000000000000000000000000000000000000000000000000000000000000000000000000000000000000000000000001EFEB8
:3C4CE000000000000000000000000000000000000000000000000000000000000000000000000000000000000000000000000000000000000000000000001EFE7C
:3C4D1C00000000000000000000000000000000000000000000000000000000000000000000000000000000000000000000000000000000000000000000001EFE3F
:3C4D5800000000000000000000000000000000000000000000000000000000000000000000000000000000000000000000000000000000000000000000001EFE03
:3C4D9400000000000000000000000000000000000000000000000000000000000000000000000000000000000000000000000000000000000000000000001EFEC7
:3C4DD000000000000000000000000000000000000000000000000000000000000000000000000000000000000000000000000000000000000000000000001EFE8B
:3C4E0C00000000000000000000000000000000000000000000000000000000000000000000000000000000000000000000000000000000000000000000001EFE4E
:3C4E4800000000000000000000000000000000000000000000000000000000000000000000000000000000000000000000000000000000000000000000001EFE12
:3C4E8400000000000000000000000000000000000000000000000000000000000000000000000000000000000000000000000000000000000000000000001EFED6
:3C4EC000000000000000000000000000000000000000000000000000000000000000000000000000000000000000000000000000000000000000000000001EFE9A
:3C4EFC00000000000000000000000000000000000000000000000000000000000000000000000000000000000000000000000000000000000000000000001EFE5E
:3C4F3800000000000000000000000000000000000000000000000000000000000000000000000000000000000000000000000000000000000000000000001EFE21
:3C4F7400000000000000000000000000000000000000000000000000000000000000000000000000000000000000000000000000000000000000000000001EFEE5
:3C4FB000000000000000000000000000000000000000000000000000000000000000000000000000000000000000000000000000000000000000000000001EFEA9
:3C4FEC00000000000000000000000000000000000000000000000000000000000000000000000000000000000000000000000000000000000000000000001EFE6D
:3C502800000000000000000000000000000000000000000000000000000000000000000000000000000000000000000000000000000000000000000000001EFE30
:3C506400000000000000000000000000000000000000000000000000000000000000000000000000000000000000000000000000000000000000000000001EFEF4
:3C50A000000000000000000000000000000000000000000000000000000000000000000000000000000000000000000000000000000000000000000000001EFEB8
:3C50DC00000000000000000000000000000000000000000000000000000000000000000000000000000000000000000000000000000000000000000000001EFE7C
:3C511800000000000000000000000000000000000000000000000000000000000000000000000000000000000000000000000000000000000000000000001EFE3F
:3C515400000000000000000000000000000000000000000000000000000000000000000000000000000000000000000000000000000000000000000000001EFE03
:3C519000000000000000000000000000000000000000000000000000000000000000000000000000000000000000000000000000000000000000000000001EFEC7
:3C51CC00000000000000000000000000000000000000000000000000000000000000000000000000000000000000000000000000000000000000000000001EFE8B
:3C520800000000000000000000000000000000000000000000000000000000000000000000000000000000000000000000000000000000000000000000001EFE4E
:3C524400000000000000000000000000000000000000000000000000000000000000000000000000000000000000000000000000000000000000000000001EFE12
:3C528000000000000000000000000000000000000000000000000000000000000000000000000000000000000000000000000000000000000000000000001EFED6
:3C52BC00000000000000000000000000000000000000000000000000000000000000000000000000000000000000000000000000000000000000000000001EFE9A
:3C52F800000000000000000000000000000000000000000000000000000000000000000000000000000000000000000000000000000000000000000000001EFE5E
:3C533400000000000000000000000000000000000000000000000000000000000000000000000000000000000000000000000000000000000000000000001EFE21
:3C537000000000000000000000000000000000000000000000000000000000000000000000000000000000000000000000000000000000000000000000001EFEE5
:3C53AC00000000000000000000000000000000000000000000000000000000000000000000000000000000000000000000000000000000000000000000000FFFB7
:3C53E800000000000000000000000000000000000000000000000000000000000000000000000000000000000000000000000000000000000000000000001EFE6D
:3C542400000000000000000000000000000000000000000000000000000000000000000000000000000000000000000000000000000000000000000000001EFE30
:3C546000020000000000000000000000000000000000000000000000000000000000000000000000000000000000000000000000000000000000000000003EFED2
:3C549C00020000000000000000000000000000000000000000000000000000000000000000000000000000000000000000000000000000000000000000002FFFA4
:3C54D800000000000000000000000000000000000000000000000000000000000000000000000000000000000000000000000000000000000000000000000FFF8A
:3C551400020000000000000000000000000000000000000000000000000000000000000000000000000000000000000000000000000000000000000000002FFF2B
:3C555000020000000000000000000000000000000000000000000000000000000000000000000000000000000000000000000000000000000000000000002FFFEF
:3C558C00020000000000000000000000000000000000000000000000000000000000000000000000000000000000000000000000000000000000000000002FFFB3
:3C55C800000000000000000000000000000000000000000000000000000000000000000000000000000000000000000000000000000000000000000000001EFE8B
:3C560400000000000000000000000000000000000000000000000000000000000000000000000000000000000000000000000000000000000000000000001EFE4E
:3C564000020000000000000000000000000000000000000000000000000000000000000000000000000000000000000000000000000000000000000000003EFEF0
:3C567C00020000000000000000000000000000000000000000000000000000000000000000000000000000000000000000000000000000000000000000002FFFC2
:3C56B800020000000000000000000000000000000000000000000000000000000000000000000000000000000000000000000000000000000000000000002FFF86
:3C56F400020000000000000000000000000000000000000000000000000000000000000000000000000000000000000000000000000000000000000000003EFE3C
:3C573000020000000000000000000000000000000000000000000000000000000000000000000000000000000000000000000000000000000000000000003EFEFF
:3C576C00000000000000000000000000000000000000000000000000000000000000000000000000000000000000000000000000000000000000000000001EFEE5
:3C57A800000000000000000000000000000000000000000000000000000000000000000000000000000000000000000000000000000000000000000000001EFEA9
:3C57E400000000000000000000000000000000000000000000000000000000000000000000000000000000000000000000000000000000000000000000001EFE6D
:3C582000020000000000000000000000000000000000000000000000000000000000000000000000000000000000000000000000000000000000000000002FFF1C
:3C585C00020000000000000000000000000000000000000000000000000000000000000000000000000000000000000000000000000000000000000000002FFFE0
:3C589800000000000000000000000000000000000000000000000000000000000000000000000000000000000000000000000000000000000000000000001EFEB8
:3C58D400020000000000000000000000000000000000000000000000000000000000000000000000000000000000000000000000000000000000000000002FFF68
:3C591000020000000000000000000000000000000000000000000000000000000000000000000000000000000000000000000000000000000000000000002FFF2B
:3C594C00020000000000000000000000000000000000000000000000000000000000000000000000000000000000000000000000000000000000000000002FFFEF
:3C598800000000000000000000000000000000000000000000000000000000000000000000000000000000000000000000000000000000000000000000001EFEC7
:3C59C400000000000000000000000000000000000000000000000000000000000000000000000000000000000000000000000000000000000000000000001EFE8B
:3C5A0000020000000000000000000000000000000000000000000000000000000000000000000000000000000000000000000000000000000000000000003EFE2C
:3C5A3C00020000000000000000000000000000000000000000000000000000000000000000000000000000000000000000000000000000000000000000002FFFFE
:3C5A7800020000000000000000000000000000000000000000000000000000000000000000000000000000000000000000000000000000000000000000002FFFC2
:3C5AB400020000000000000000000000000000000000000000000000000000000000000000000000000000000000000000000000000000000000000000003EFE78
:3C5AF00002000000000000000000000000000000000000000000000000000080010000000000000000000000000000000000000000000000000000000000A6FF52
:3C5B2C00020000000000000000000000000000000000000000000000000000000000000000000000000000000000000000000000000000000000000000003EFEFF
:3C5B6800000000000000000000000000000000000000000000000000000000000000000000000000000000000000000000000000000000000000000000001EFEE5
:3C5BA400000000000000000000000000000000000000000000000000000000000000000000000000000000000000000000000000000000000000000000001EFEA9
:3C5BE000020000000000000000000000000000000000000000000000000000000000000000000000000000000000000000000000000000000000000000002FFF59
:3C5C1C00020000000000000000000000000000000000000000000000000000000000000000000000000000000000000000000000000000000000000000002FFF1C
:3C5C5800020000000000000000000000000000000000000000000000000000000000000000000000000000000000000000000000000000000000000000003EFED2
:3C5C9400020000000000000000000000000000000000000000000000000000000000000000000000000000000000000000000000000000000000000000002FFFA4
:3C5CD0000A080000000000000000000000000000000000000000000000000000000000000000000000000000000000000000000000000000000000000000A7FFE0
:3C5D0C0002900000000000000000000000000000000000000000000000000000000000000000000000000000000000000000000000000000000000000000BFFF0B
:3C5D4800000000000000000000000000000000000000000000000000000000000000000000000000000000000000000000000000000000000000000000001EFE03
:3C5D840000800600000000000000000000000000000000000000000000000000000000000000000000000000000000000000000000000000000000000000F8FE67
:3C5DC00002A00600000000000000000000000000000000000000000000000000000000000000000000000000000000000000000000000000000000000000F8FE09
:3C5DFC0002800000000000000000000000000000000000000000000000000000000000000000000000000000000000000000000000000000000000000000AFFF3B
:3C5E3800020000000000000000000000000000000000000000000000000000000000000000000000000000000000000000000000000000000000000000002FFFFE
:3C5E74000200060000000000000000000000000000000000000000000000000000000000000000000000000000000000000000000000000000000000000058FE94
:3C5EB0000200060000000000000000000000000000000000000000000000000000000000000000000000000000000000000000000000000000000000000058FE58
:3C5EEC00008000000000000000000000000000000000000000000000000000000000000000000000000000000000000000000000000000000000000000008FFF6C
:3C5F2800000000000000000000000000000000000000000000000000000000000000000000000000000000000000000000000000000000000000000000001EFE21
:3C5F640000800600000000000000000000000000000000000000000000000000000000000000000000000000000000000000000000000000000000000000F8FE85
:3C5FA00002800000000000000000000000000000000000000000000000000000000000000000000000000000000000000000000000000000000000000000BEFE87
:3C5FDC0002B000000000000000000000000000000000000000000000000000000000000000000000000000000000000000000000000000000000000000009FFF39
:3C6018000200060000000000000000000000000000000000000000000000000000000000000000000000000000000000000000000000000000000000000049FFFC
:3C6054000000060000000000000000000000000000000000000000000000000000000000000000000000000000000000000000000000000000000000000078FE94
:3C609000000000000000000000000000000000000000000000000000000000000000000000000000000000000000000000000000000000000000000000001EFEB8
:3C60CC00008000000000000000000000000000000000000000000000000000000000000000000000000000000000000000000000000000000000000000009EFE7C
:3C610800000000000000000000000000000000000000000000000000000000000000000000000000000000000000000000000000000000000000000000001EFE3F
:3C61440000800600000000000000000000000000000000000000000000000000000000000000000000000000000000000000000000000000000000000000F8FEA3
:3C61800002800000000000000000000000000000000000000000000000000000000000000000000000000000000000000000000000000000000000000000AFFFB3
:3C61BC0002D00000000000000000000000000000000000000000000000000000000000000000000000000000000000000000000000000000000000000000FFFFD7
:3C61F8000000060000000000000000000000000000000000000000000000000000000000000000000000000000000000000000000000000000000000000078FEEF
:3C6234000200060000000000000000000000000000000000000000000000000000000000000000000000000000000000000000000000000000000000000049FFDE
:3C627000020000000000000000000000000000000000000000000000000000000000000000000000000000000000000000000000000000000000000000002FFFC2
:3C62AC00008000000000000000000000000000000000000000000000000000000000000000000000000000000000000000000000000000000000000000008FFFA8
:3C62E800000000000000000000000000000000000000000000000000000000000000000000000000000000000000000000000000000000000000000000001EFE5E
:3C63240000800600000000000000000000000000000000000000000000000000000000000000000000000000000000000000000000000000000000000000F8FEC1
:3C63600002800600000000000000000000000000000000000000000000000000000000000000000000000000000000000000000000000000000000000000D8FEA3
:3C639C0002800600000000000000000000000000000000000000000000000000000000000000000000000000000000000000000000000000000000000000C9FF75
:3C63D8000200060000000000000000000000000000000000000000000000000000000000000000000000000000000000000000000000000000000000000049FF39
:3C641400000000000000000000000000000000000000000000000000000000000000000000000000000000000000000000000000000000000000000000001EFE30
:3C645000000000000000000000000000000000000000000000000000000000000000000000000000000000000000000000000000000000000000000000001EFEF4
:3C648C00009000000000000000000000000000000000000000000000000000000000000000000000000000000000000000000000000000000000000000009FFFA6
:3C64C8000000060000000000000000000000000000000000000000000000000000000000000000000000000000000000000000000000000000000000000078FE1C
:3C650400000000000000000000000000000000000000000000000000000000000000000000000000000000000000000000000000000000000000000000001EFE3F
:3C65400002A00600000000000000000000000000000000000000000000000000000000000000000000000000000000000000000000000000000000000000F8FE81
:3C657C00020100000000000000000000000000000000000000000000000000000000000000000000000000000000000000000000000000000000000000003FFEA3
:3C65B8000000068000800080008000800080008000800080008000800080008000800080008000800080008000800080008000800080008000800080000069FFB9
:3C65F400020000000000000000000000000000000000000000000000000000000000000000000000000000000000000000000000000000000000000000003EFE2D
:3C6630000240060000000000000000000000000000000000000000000000000000000000000000000000000000000000000000000000000000000000000018FED0
:3C666C00000000000000000000000000000000000000000000000000000000000000000000000000000000000000000000000000000000000000000000001EFED6
:3C66A800002000000000000000000000000000000000000000000000000000000000000000000000000000000000000000000000000000000000000000003EFE5A
:3C66E400000000000000000000000000000000000000000000000000000000000000000000000000000000000000000000000000000000000000000000001EFE5E
:3C672000000000000000000000000000000000000000000000000000000000000000000000000000000000000000000000000000000000000000000000001EFE21
:3C675C00000000000000000000000000000000000000000000000000000000000000000000000000000000000000000000000000000000000000000000001EFEE5
:3C679800000000000000000000000000000000000000000000000000000000000000000000000000000000000000000000000000000000000000000000001EFEA9
:3C67D400000000000000000000000000000000000000000000000000000000000000000000000000000000000000000000000000000000000000000000001EFE6D
:3C681000000000000000000000000000000000000000000000000000000000000000000000000000000000000000000000000000000000000000000000001EFE30
:3C684C00400000000000000000000000000000000000000000000000000000000100000000000000000000000000000000000000000000000000000000004AFF86
:3C688800000000000000000000000000000000000000000000000000000000000000000000000000000000000000000000000000000000000000000000001EFEB8
:3C68C400000000000000000000000000000000000000000000000000000000000000000000000000000000000000000000000000000000000000000000001EFE7C
:3C690000000000000000000000000000000000000000000000000000000000000000000000000000000000000000000000000000000000000000000000001EFE3F
:3C693C00000000000000000000000000000000000000000000000000000000000000000000000000000000000000000000000000000000000000000000001EFE03
:3C697800000000000000000000000000000000000000000000000000000000000000000000000000000000000000000000000000000000000000000000001EFEC7
:3C69B400000000000000000000000000000000000000000000000000000000000000000000000000000000000000000000000000000000000000000000001EFE8B
:3C69F000000000000000000000000000000000000000000000000000000000000000000000000000000000000000000000000000000000000000000000001EFE4F
:3C6A2C00000000000000000000000000000000000000000000000000000000000000000000000000000000000000000000000000000000000000000000001EFE12
:3C6A6800000000000000000000000000000000000000000000000000000000000000000000000000000000000000000000000000000000000000000000001EFED6
:3C6AA400000000000000000000000000000000000000000000000000000000000000000000000000000000000000000000000000000000000000000000001EFE9A
:3C6AE000000000000000000000000000000000000000000000000000000000000000000000000000000000000000000000000000000000000000000000001EFE5E
:3C6B1C00000000000000000000000000000000000000000000000000000000000000000000000000000000000000000000000000000000000000000000001EFE21
:3C6B5800000000000000000000000000000000000000000000000000000000000000000000000000000000000000000000000000000000000000000000001EFEE5
:3C6B9400000000000000000000000000000000000000000000000000000000000000000000000000000000000000000000000000000000000000000000001EFEA9
:3C6BD000000000000000000000000000000000000000000000000000000000000000000000000000000000000000000000000000000000000000000000001EFE6D
:3C6C0C00000000000000000000000000000000000000000000000000000000000000000000000000000000000000000000000000000000000000000000001EFE30
:3C6C4800000000000000000000000000000000000000000000000000000000000000000000000000000000000000000000000000000000000000000000001EFEF4
:3C6C8400000000000000000000000000000000000000000000000000000000000000000000000000000000000000000000000000000000000000000000001EFEB8
:3C6CC000000000000000000000000000000000000000000000000000000000000000000000000000000000000000000000000000000000000000000000001EFE7C
:3C6CFC00000000000000000000000000000000000000000000000000000000000000000000000000000000000000000000000000000000000000000000001EFE40
:3C6D3800000000000000000000000000000000000000000000000000000000000000000000000000000000000000000000000000000000000000000000001EFE03
:3C6D7400000000000000000000000000000000000000000000000000000000000000000000000000000000000000000000000000000000000000000000001EFEC7
:3C6DB000000000000000000000000000000000000000000000000000000000000000000000000000000000000000000000000000000000000000000000001EFE8B
:3C6DEC00000000000000000000000000000000000000000000000000000000000000000000000000000000000000000000000000000000000000000000001EFE4F
:3C6E2800000000000000000000000000000000000000000000000000000000000000000000000000000000000000000000000000000000000000000000001EFE12
:3C6E6400000000000000000000000000000000000000000000000000000000000000000000000000000000000000000000000000000000000000000000001EFED6
:3C6EA000000200000000000000000000000000000000000000000000000000000000000000000000000000000000000000000000000000000000000000001CFE9A
:3C6EDC00020000000000000000000000000000000000000000000000000000000000000000000000000000000000000000000000000000000000000000002FFF4A
:3C6F1800000000000000000000000000000000000000000000000000000000000000000000000000000000000000000000000000000000000000000000001EFE21
:3C6F5400000000000000000000000000000000000000000000000000000000000000000000000000000000000000000000000000000000000000000000001EFEE5
:3C6F9000000000000000000000000000000000000000000000000000000000000000000000000000000000000000000000000000000000000000000000001EFEA9
:3C6FCC00000000000000000000000000000000000000000000000000000000000000000000000000000000000000000000000000000000000000000000001EFE6D
:3C700800000000000000000000000000000000000000000000000000000000000000000000000000000000000000000000000000000000000000000000001EFE30
:3C704400000000000000000000000000000000000000000000000000000000000000000000000000000000000000000000000000000000000000000000001EFEF4
:3C708000000000000000000000000000000000000000000000000000000000000000000000000000000000000000000000000000000000000000000000001EFEB8
:3C70BC00000000000000000000000000000000000000000000000000000000000000000000000000000000000000000000000000000000000000000000001EFE7C
:3C70F800000000000000000000000000000000000000000000000000000000000000000000000000000000000000000000000000000000000000000000001EFE40
:3C713400000000000000000000000000000000000000000000000000000000000000000000000000000000000000000000000000000000000000000000001EFE03
:3C717000020000000000000000000000000000000000000000000000000000000000000000000000000000000000000000000000000000000000000000002FFFB3
:3C71AC00020000000000000000000000000000000000000000000000000000000000000000000000000000000000000000000000000000000000000000002FFF77
:3C71E800020000000000000000000000000000000000000000000000000000000000000000000000000000000000000000000000000000000000000000003EFE2D
:3C722400000000000000000000000000000000000000000000000000000000000000000000000000000000000000000000000000010000000000000000001FFF0F
:3C7260000000000000000000000000000000000000000000000000000000000000000000000000000000000000000000000000800000000000000000000007FF6C
:3C729C000000000000000000000000000000000000000000000000901600000000000000000000000000000000000000000000000000000000000000000066FEAC
:3C72D800000000000000000000000000000000000000000000000000060000000000000000000000000000000000000000000000000000000000000000007EFEF8
:3C731400000000000000000000000000000000000000000000000000000000000000000000000000000000000000000000000000000000000000000000001EFE21
:3C7350000200000000000000000000000000000000000000000000A02000000000000000000000000000000000000000000000000000000000000000000007FF39
:3C738C00020000000000000000000000000000000000000000000000060000000000000000000000000000000000000000000000000000000000000000004FFF6F
:3C73C800020000000000000000000000000000000000000000000000060000000000000000000000000000000000000000000000000000000000000000005EFE25
:3C7404000000000000000000000000000000000000000000000000800600000000000000000000000000000000000000000000000000000000000000000067FF60
:3C744000000000000000000000000000000000000000000000000000060000000000000000000000000000000000000000000000000000000000000000006FFF9C
:3C747C000000000000000000000000000000000000000000000000D00600000000000000000000000000000000000000000000000000000000000000000062FF9D
:3C74B800000000000000000000000000000000000000000000000000060000000000000000000000000000000000000000000000000000000000000000007EFE16
:3C74F400000000000000000000000000000000000000000000000000040000000000000000000000000000000000000000000000000000000000000000005EFEFC
:3C7530000200000000000000000000000000000000000000000000803600000000000000000000000000000000000000000000000000000000000000000065FE04
:3C756C00020000000000000000000000000000000000000000000010060000000000000000000000000000000000000000000000000000000000000000005FFE6E
:3C75A800000000000000000000000000000000000000000000000000060000000000000000000000000000000000000000000000000000000000000000007EFE25
:3C75E4000200000000000000000000000000000000000000000000800600000000000000000000000000000000000000010000000000000000000000000047FE9D
:3C76200002000000000000000000000000000000000000000000004016020000000000000000000000000000000000800000000000000000000000000000C9FE8D
:3C765C000000000000000000000000000000000000000000000000800400008806000000000000000000000000000000000000000000000000000000000058FE8A
:3C7698000000000000000000000000000000000000000000000000000400000006000000000000000000000000000000000000000000000000000000000058FE56
:3C76D40000000000000000000000000000000000000000000000008002000080000000000000000000000000000000000000000000000000000000000000BEFEBC
:3C771000020000000000000000000000000000000000000000000080020000C0300000000000000000000000000000000000000000000000000000000000FBFFCF
:3C774C0002000000000000000000000000000000000000000000008004000080060000000000000000000000000000000000000000000000000000000000E9FF0D
:3C7788000200000000000000000000000000000000000000000000000200000006000000000000000000000000000000000000000000000000000000000018FEA5
:3C77C40000000000000000000000000000000000000000000000000002000080000000000000000000000000000000000000000001000000000000000000B7FF50
:3C7800000000000000000000000000000000000000000000000000003400000000000000000000000000000000000000000000800000000000000000000065FE35
:3C783C000000000000000000000000000000000000000000000000800000000000000000000000000000000000000000000000000000000000000000000016FE7C
:3C787800000000000000000000000000000000000000000000000000000000000000000000000000000000000000000000000000000000000000000000001EFEB8
:3C78B4000000000000000000000000000000000000000000000000800600000000000000000000000000000000000000000000000000000000000000000076FE9E
:3C78F0000200000000000000000000000000000000000000000000800000000000000000000000000000000000000000000000000000000000000000000027FFB4
:3C792C000200000000000000000000000000000000000000000000900000000000000000000000000000000000000000000000000000000000000000000037FE58
:3C796800020000000000000000000000000000000000000000000000060000000000000000000000000000000000000000000000000000000000000000005EFE7F
:3C79A400000000000000000000000000000000000000000000000000060000000000000000000000000000000000000000000000000000000000000000006FFF33
:3C79E000000000000000000000000000000000000000000000000020000000000000000000000000000000000000000000000000000000000000000000000DFF3F
:3C7A1C00000000000000000000000000000000000000000000000080000000000000000000000000000000000000000000000000000000000000000080000FFF20
:3C7A5800000000000000000000000000000000000000000000000000000000000000000000000000000000000000000000000000000000000000000000001EFED6
:3C7A94000000000000000000000000000000000000000000000000800600000000000000000000000000000000000000000000000000000000000000000076FEBC
:3C7AD0000200000000000000000000000000000000000000000000800000000000000000000000000000000000000000000000000000000000000000002005FFD4
:3C7B0C000200000000000000000000000000000000000000000000B000000000000000000000000000000000000000000000000000000000000000000048F1FE54
:3C7B4800000000000000000000000000000000000000000000000000060000000000000000000000000000000000000000000000000000000000000000006FFF8D
:3C7B8400020000000000000000000000000000000000000000000000060000000000000000000000000000000000000000000000000000000000000000004FFF6F
:3C7BC00002000000000000000000000000000000000000000000000000800100000000000000000000000000000000000000000000000000000000000000BEFF49
:3C7BFC0000000000000000000000000000000000000000000000008000000084060000000000000000000000000000000000000000000000000000000000D8FE6D
:3C7C3800000000000000000000000000000000000000000000000000000000000000000000000000000000000000000000000000000000000000000000001EFEF4
:3C7C740000000000000000000000000000000000000000000000008006000080040000000000000000000000000000000000000000000000000000000000FAFED2
:3C7CB000020000000000000000000000000000000000000000000080000000A00A0400000000000000000000000000000000000000000000000000000000C3FFA6
:3C7CEC000200000000000000000000000000000000000000000000D0000000D0000000000000000000000000000000000000000000000000000000000000FFFFBC
:3C7D28000000000000000000000000000000000000000000000000000600000006000000000000000000000000000000000000000000000000000000000078FE9D
:3C7D640002000000000000000000000000000000000000000000000006000080000000000000000000000000000000000000000000000000000000000000C7FF95
:3C7DA0000200000000000000000000000000000000000000000000000000000036000000000000000000000000000000000000000000000000000000000019FF57
:3C7DDC00000000000000000000000000000000000000000000000080000000C4000000000000000000000000000000000000000000000000000080A08600CDFFB5
:3C7E1800000000000000000000000000000000000000000000000000000000000600000000000000000000000000000000000000000000000000000006007EFEA6
:3C7E540000000000000000000000000000000000000000000000008006000000000000000000000000000000000000000000000000000000000000800200D4FE18
:3C7E900002000000000000000000000000000000000000000000008006000080060000000000000000000000000000000000000000000000000000800A30C1FE2F
:3C7ECC0002000000000000000000000000000000000000000000008006000022000000000000000000000000000000000000000000000000000000800808CDFF74
:3C7F08000200000000000000000000000000000000000000000000000600000006000000000000000000000000000000000000000000000000000000000049FFE7
:3C7F44000000000000000000000000000000000000000000000000000000008000000000000000000000000000000000000000000000000000000080020025FFDB
:3C7F80000000000000000000000000000000000000000000000000000000000006000000000000000000000000000000000000000000000000000000044108FE74
:3C7FBC0000000000000000000000000000000000000000000000000000000084060000000000000000000000000000000000000000000000000040808E00E3FFCF
:3C7FF8000000000000000000000000000000000000000000000000000000000000000000000000000000000000000000000000000000000000000000060078FED1
:3C80340000000000000000000000000000000000000000000000000000000000060000000000000000000000000000000000000000000000000000800600FEFE88
:3C807000020000000000000000000000000000000000000000000000000000A0000000000000000000000000000000000000000000000000000000A0002117FF5B
:3C80AC000200000000000000000000000000000000000000000000000800000406000000000000000000000000000000000000000000000000000088001061FE8D
:3C80E80002800080008000800080008000800080008000800080000000800080068000800080008000800080008000800080008000800080008000800600C7FF08
:3C8124000000000000000000000000000000000000000000000000000000000006000000000000000000000000000000000000000000000000000000000009FF11
:3C81600000800100000000000000000000000000000000000000000020000040060000000000000000000000000000000000000000000000000000400040FAFF83
:3C819C000000000000000000000000000000000000000000000000800001000000000000000000000000000000000000000000000000000000000000000006FF21
:3C81D8000000000000000000000000000000000000000000000000080000000800000000000000000000000000000000000000000000000000000020000036FE07
:3C821400000000000000000000000000000000000000000000000000000000000000000000000000000000000000000000000000000000000000000000001EFE12
:3C825000000000000000000000000000000000000000000000000000000000000000000000000000000000000000000000000000000000000000000000001EFED6
:3C828C00000000000000000000000000000000000000000000000000000000100400000000000000000000000000000000000000000000000000000000001AFF89
:3C82C800000000000000000000000000000000000000000000000000000000000000000000000000000000000000000000000000000000000000000000001EFE5E
:3C830400000000000000000000000000000000000000000000000000000000000000000000000000000000000000000000000000000000000000000000001EFE21
:3C834000000000000000000000000000000000000000000000000000000000000000000000000000000000000000000000000000010000000000080000008EFE6C
:3C837C00000000000000000000000000000000000000000000000000000000000000000000000000000000000000000000000000000000000000000000001EFEA9
:3C83B800000002000000000000000000000000000000000000000000000000020000000000000000000000000000000000000000000000000000000000001CFE6B
:3C83F400000000000000000000000000000000000000000000000000000000000000000000000000000000000000000001000000000000000000000000010EFF3E
:3C843000000000000000000000000000000000000000000000000000000000000000000000000000000000000000000000000000000000000000000000001EFEF4
:3C846C000000000000000000000000000000000000000000000000000200000800080000000000000000000000000000000000000000000000000000000036FE8E
:3C84A800000000000000000000000000000000000000000000000000000000000000000000000000000000000000000000000000000000000000000000001EFE7C
:3C84E400000000000000000000000000000000000000000000000000000000000000000000000000000000000000000000000000000000000000000000001EFE40
:3C8520000000000000000000000000000000000000000000000000800102004000000000000000000000000000000000000000000000000000000000000040FE1E
:3C855C00000000000000000000000000000000000000000000000000000000000000000000000000000000000000000000000000000000000000000000001EFEC7
:3C859800000000000000000000000000000000000000000000000000000000000000000000000000000000000000000000000000000000000000000000001EFE8B
:3C85D400000000000000000000000000000000000000000000000000000000000000000000000000000000000000000000000000000000000000000000001EFE4F
:3C861000000000000000000000000000000000000000000000000000000000000000000000000000000000000000000000000000000000000000000000001EFE12
:3C864C00000000000000000000000000000000000000000000000000000000000000000000000000000000000000000000000000000000000000000000001EFED6
:3C868800000000000000000000000000000000000000000000000000000000000000000000000000000000000000000000000000000000000000000000001EFE9A
:3C86C400000000000000000000000000000000000000000000000000000000000000000000000000000000000000000000000000000000000000000000001EFE5E
:3C870000000000000000000000000000000000000000000000000000000000000000000000000000000000000000000000000000000000000000000000001EFE21
:3C873C00000000000000000000000000000000000000000000000000000000000000000000000000000000000000000000000000000000000000000000001EFEE5
:3C877800000000000000000000000000000000000000000000000000000000000000000000000000000000000000000000000000000000000000000000001EFEA9
:3C87B4000000000000000000000000000000000000000000000000000000000000000000000000000000000000000000000000080000000000001000000096FFDC
:3C87F000000000000000000000000000000000000000000000000000000000000000000000000000000000000000000000000000000000000000000000001EFE31
:3C882C000000000000000000000000000000000000000000000000000000001000000000000000000000000000000000000000000000000000000000008096FFEB
:3C886800000000000000000000000000000000000000000000000000000000000000000000000000000000000000000000000000000000000000000000001EFEB8
:3C88A400000000000000000000000000000000000000000000000000000000000000000000000000000000000000000000000000000000000000000000001EFE7C
:3C88E000000000000000000000000000000000000000000000000000000000000000000000000000000000000000000000000000000000000000000000001EFE40
:3C891C000000000000000000000000000000000000000000000000000000200000000000000000000000000000000000000000000000000000000000080094FE65
:3C895800000000000000000000000000000000000000000000000000000000000000000000000000000000000000000000000000000000000000000000001EFEC7
:3C899400000000000000000000000000000000000000000000000000000000200000000000000000000000000000000000000000000000000000000000003CFE4D
:3C89D000000000000000000000000000000000000000000000000000000000000000000000000000000000000000000000000000000000000000000000001EFE4F
:3C8A0C00000000000000000000000000000000000000000000000000000000000000000000000000000000000000000000A11600008000000000000080002BFF4D
:3C8A48000000000000000000000000000000000000000000000000000000000000000000000000000000000000000000000006000000000000000000000018FED6
:3C8A840000000000000000000000000000000000000000000000000000000000000000000000000000000000000000000000060000800200000000000000BAFE76
:3C8AC0000200000000000000000000000000000000000000000000000000000000000000000000000000000000000000008026000080020000000000002001FF30
:3C8AFC000200000000000000000000000000000000000000000000000000000000000000000000000000000000000000004206000080040000000000000809FF60
:3C8B3800020000000000000000000000000000000000000000000000000000000000000000000000000000000000000000000200000002000000000000000FFFED
:3C8B740000000000000000000000000000000000000000000000000000000000000000000000000000000000000000000080060000000200000000000000A3FF9B
:3C8BB000000000000000000000000000000000000000000000000000000000000000000000000000000000000000000000000E8201004C00000000000040A6FEC8
:3C8BEC00000000000000000000000000000000000000000000000000000000000000000000000000808006000000000000D00200008000000000000000003EFFB8
:3C8C2800000000000000000000000000000000000000000000000000000000000000000000000000000006000000000000000600000000000000000000007EFE88
:3C8C640000000000000000000000000000000000000000000000000000000000000000000000000000000600000000000000060000800200000000000000DCFE6C
:3C8CA00002000000000000000000000000000000000000000000000000000000000000000000000000C00600000000000080560000800200000000000000F5FF84
:3C8CDC0002000000000000000000000000000000000000000000000000000000000000000000000000000000000000000010060000800400000000000000EDFED5
:3C8D1800000000000000000000000000000000000000000000000000000000000000000000000000000000000000000000000600000002000000000000003AFEDF
:3C8D54000200000000000000000000000000000000000000000000000000000000000000000000000080000000000000008006000000020000000000000003FFD7
:3C8D900002000000000000000000000000000000000000000000000000000000000000000000000000000000000000000040160200002C0000000000000091FF91
:3C8DCC00000000000000000000000000000000000000000000000000000000000000000000000000000000000000000000C40600008000000000000080000DFF95
:3C8E08000000000000000000000000000000000000000000000000000000000000000000000000000000000000000000000006000000000000000000000018FE12
:3C8E440000000000000000000000000000000000000000000000000000000000000000000000000000000000000000000000060000800200000000000000BAFEB2
:3C8E8000020000000000000000000000000000000000000000000000000000000000000000000000000000000000000000804E000080020000000000002069FFDC
:3C8EBC0002000000000000000000000000000000000000000000000000000000000000000000000000000000000000000008040000800C00000000000010E7FEEB
:3C8EF800000000000000000000000000000000000000000000000000000000000000000000000000000000000000000000000600000002000000000000002BFF0C
:3C8F34000200000000000000000000000000000000000000000000000000000000000000000000000000000000000000008006000000020000000000000083FFF5
:3C8F7000020000000000000000000000000000000000000000000000000000000000000000000000000000000000000000402E000000240000000000004056FE9D
:3C8FAC00020000000000000000000000000000000000000000000000000000000000000000000000000000000000000000800400008000000000000080002BFFD9
:3C8FE800000000000000000000000000000000000000000000000000000000000000000000000000000000000000000000000400000000000000000000001AFE31
:3C9024000000000000000000000000000000000000000000000000000000000000000000000000000000000000000000008002000080020000000000000036FED8
:3C9060000200000000000000000000000000000000000000000000000000000000000000000000000000000000000000008002000080020000000000002025FF8A
:3C909C000200000000000000000000000000000000000000000000000000000000000000000000000000000000000000008014000080140000000000005023FFFC
:3C90D800020000000000000000000000000000000000000000000000000000000000000000000000000000000000000000000200000002000000000000000FFF48
:3C911400020000000000000000000000000000000000000000000000000000000000000000000000000000000000000001000200000002000000000000000FFE0B
:3C91500002000000000000000000000000000000000000000000000000000000000000000000000000000000000000800000248001002400000000000000C4FED6
:3C918C000000000000000000000000000000000000000000000000000000000000000000000000000000000000000000008000000080000000000000000016FE93
:3C91C800000000000000000000000000000000000000000000000000000000000000000000000000000000000000000000000000000000000000000000001EFE4F
:3C9204000000000000000000000000000000000000000000000000000000000000000000000000000000000000000000008002000080020000000000000036FEF6
:3C9240000200000000000000000000000000000000000000000000000000000000000000000000000000000000000000008002000080020000000000000007FFE6
:3C927C000200000000000000000000000000000000000000000000000000000000000000000000000000000000000000008004000080040000000000000067FF46
:3C92B800000000000000000000000000000000000000000000000000000000000000000000000000000000000000000000000200000002000000000000003EFE3A
:3C92F400020000000000000000000000000000000000000000000000000000000000000000000000000000000000000000000200000002000000000000000FFF2A
:3C933000020000000000000000000000000000000000000000000000000000000000000000000000000000000000000000003400000034000000000000004DFE4C
:3C936C000200000000000000000000000000000000000000000000000000000000000000000000000000000000000000008000000080000000000000000036FE8F
:3C93A800000000000000000000000000000000000000000000000000000000000000000000000000000000000000000000000000000000000000000000001EFE6D
:3C93E4000000000000000000000000000000000000000000000000000000000000000000000000000000000000000000008006000080060000000000000076FECD
:3C9420000200000000000000000000000000000000000000000000000000000000000000000000000000000000000000008000000080000000000000000027FFE8
:3C945C000200000000000000000000000000000000000000000000000000000000000000000000000000000000000000009000000090000000000000000037FE7D
:3C949800020000000000000000000000000000000000000000000000000000000000000000000000000000000000000000000600000006000000000000005EFE2E
:3C94D400020000000000000000000000000000000000000000000000000000000000000000000000000000000000000000000600000006000000000000004FFF00
:3C951000020000000000000000000000000000000000000000000000000000000000000000000000000000000000000000200000002000000000000000002DFFB1
:3C954C0000000000000000000000000000000000000000000000000000000000000000000000000000000000000000000080000000800000000000C11600B0FE5E
:3C9588000000000000000000000000000000000000000000000000000000000000000000000000000000000000000000000000000000000000000000060078FE2B
:3C95C40000000000000000000000000000000000000000000000000000000000000000000000000000000000000000000080060000800600000000800200D4FE0B
:3C9600000200000000000000000000000000000000000000000000000000000000000000000000000000000000000000008000000080000000000080021085FE17
:3C963C00020000000000000000000000000000000000000000000000000000000000000000000000000000000000000000B0000000B00000000000800000B5FE5D
:3C967800000000000000000000000000000000000000000000000000000000000000000000000000000000000000000000000600000006000000000000007EFE2E
:3C96B40002000000000000000000000000000000000000000000000000000000000000000000000000000000000000000000060000000600000000800200EDFFFE
:3C96F00002000000000000000000000000000000000000000000000000800100000000000000000000000000000000000000008001000000000000000C016BFEC4
:3C972C000000000000000000000000000000000000000000000000000000000000000000000000000000000000A40E000080000000800000000000D002004AFE35
:3C976800000000000000000000000000000000000000000000000000000000000000000000000000000000000000060000000000000000000000000002005CFE63
:3C97A40000000000000000000000000000000000000000000000000000000000000000000000000000000000000006000080060000800600000000800600F0FE03
:3C97E00002000000000000000000000000000000000000000000000000000000000000000000000000000000008006020080000000800000000000800E0133FF02
:3C981C00020000000000000000000000000000000000000000000000000000000000000000000000000000008040040000D0000000D0000000000080100067FFB4
:3C985800000000000000000000000000000000000000000000000000000000000000000000000000000000000000060000000600000006000000000000001EFEA6
:3C98940002000000000000000000000000000000000000000000000000000000000000000000000000000000008006000000060001000600000000800400F3FF8D
:3C98D000020000000000000000000000000000000000000000000000000000000000000000000000000000000000160800000080000000000000000002042DFE8B
:3C990C0000000000000000000000000000000000000000000000000000000000000000000000000000000000000000000080000000800000000000848600EDFF29
:3C9948000000000000000000000000000000000000000000000000000000000000000000000000000000000000000000000000000000000000000000060078FE67
:3C99840000000000000000000000000000000000000000000000000000000000000000000000000000000000000000000080060000800600000000800200D4FE47
:3C99C00002000000000000000000000000000000000000000000000000000000000000000000000000000000000000000080000000800600000000A00A3069FE22
:3C99FC0002000000000000000000000000000000000000000000000000000000000000000000000000000000000000000090000000800600000000800030E3FF85
:3C9A3800000000000000000000000000000000000000000000000000000000000000000000000000000000000000000000000600000006000000000000006FFF78
:3C9A7400020000000000000000000000000000000000000000000000000000000000000000000000000000000000000000000600000000000000008002008BFFA2
:3C9AB00002000000000000000000000000000000000000000000000000000000000000000000000000000000000000000040000000000000000000000C01A6FE87
:3C9AEC00000000000000000000000000000000000000000000000000000000000000000000000000000000000000000000900600000000000000008806007EFF9D
:3C9B28000000000000000000000000000000000000000000000000000000000000000000000000000000000000000000000006000000000000000000000018FEE5
:3C9B640000000000000000000000000000000000000000000000000000000000000000000000000000000000000000000000060000000000000000800600FEFE3D
:3C9BA000020000000000000000000000000000000000000000000000000000000000000000000000000000000000000000A0360000000000000000C00E018DFF56
:3C9BDC0002000000000000000000000000000000000000000000000000000000000000000000000000000000000000000030000000000000000000A20000AFFECC
:3C9C18000080008000800080008000800080008000800080008000800080008000800080008000800080008000800080008006800000008000800080000018FE74
:3C9C54000200000000000000000000000000000000000000000000000000000000000000000000000000000000000000000006000000000000000000000029FFA4
:3C9C9000020000000000000000000000000000000000000000000000000000000000000000000000000000000000000000000E0400000804000000000600CBFFA8
:3C9CCC000000000000000000000000000000000000000000000000000000000000000000000000000000000000000000008000010080000100000000000006FF55
:3C9D0800000000000000000000000000000000000000000000000000000000000000000000000000000000000000000000200000002000000000002000003CFE85
:3C9D4400000000000000000000000000000000000000000000000000000000000000000000000000000000000000000000000000000000000000000000001EFEC7
:3C9D8000000000000000000000000000000000000000000000000000000000000000000000000000000000000000000000000000000000000000000000001EFE8B
:3C9DBC0000000000000000000000000000000000000000000000000000000000000000000000000000000000000000000000000800000400000000000000D2FE8F
:3C9DF800000000000000000000000000000000000000000000000000000000000000000000000000000000000020000000000000000002000000000000003EFED1
:3C9E3400000000000000000000000000000000000000000000000000000000000000000000000000000000000000000000000000000000000000000000001EFED6
:3C9E7000000000000000000000000000000000000000000000000000000000000000000000000000000000000000000000000000000000000000000000001EFE9A
:3C9EAC00000000000000000000000000000000000000000000000000000000000000000000000000000000000000000001000000000000000000000020001CFF3E
:3C9EE800000000000000000000000000000000000000000000000000000000000000000000000000000000000000000000000000000000000000000000001EFE22
:3C9F2400000000000000000000000000000000000000000000000000000000000000000000000000000000000000000000000000000000000000000000001EFEE5
:3C9F6000000000000000000000000000000000000000000000000000000000000000000000000000000000000000000000000000010000000000000000404AFE3C
:3C9F9C00000000000000000000000000000000000000000000000000000000000000000000000000000000000000000000000000000000000000000000001EFE6D
:3C9FD80000000000000000000000000000000000000000000000000000000000000000000000000000000000200000000000000000800000000000000000BEFEF1
:3CA01400000000000000000000000000000000000000000000000000000000000000000000000000000000000000000000000000000000000000000000001EFEF4
:3CA05000000000000000000000000000000000000000000000000000000000000000000000000000000000000000000000000002000001000000000000003CFF96
:3CA08C000000000000000000000000000000000000000000000000000000000000000000000000000000000000000000000008000000400000000000000012FE40
:3CA0C800000000000000000000000000000000000000000000000000000000000000000000000000000000000000000000000000000000000000000000001EFE40
:3CA10400000000000000000000000000000000000000000000000000000000000000000000000000000000000000002000000000000010000000000000002EFFC2
:3CA14000000000000000000000000000000000000000000000000000000000000000000000000000000000000000000000000000000000000000000000001EFEC7
:3CA17C00000000000000000000000000000000000000000000000000000000000000000000000000000000000000000000000000000000000000000000001EFE8B
:3CA1B800000000000000000000000000000000000000000000000000000000000000000000000000000000000000000000000000000000000000000000001EFE4F
:3CA1F400000000000000000000000000000000000000000000000000000000000000000000000000000000000000000000000000000000000000000000001EFE13
:3CA23000000000000000000000000000000000000000000000000000000000000000000000000000000000000000000000000000000000000000000000001EFED6
:3CA26C00000000000000000000000000000000000000000000000000000000000000000000000000000000000000000000000000000000000000000000001EFE9A
:3CA2A800000000000000000000000000000000000000000000000000000000000000000000000000000000000000000000000000080000000000000400009AFED6
:3CA2E400000000000000000000000000000000000000000000000000000000000000000000000000000000000000000000000000000000000000000000001EFE22
:3CA320000000000000000000000000000000000000000000000000000000000000000000000000000000000000400000001000002000000000000001000028FE6A
:3CA35C00000000000000000000000000000000000000000000000000000000000000000000000000000000000000000000001000000000000000000000000EFEA9
:3CA39800000000000000000000000000000000000000000000000000000000000000000000000000000000000000000000000000000000000000000000001EFE6D
:3CA3D400000000000000000000000000000000000000000000000000000000000000000000000000000000000000000000000002000000000000004000007CFE91
:3CA41000000000000000000000000000000000000000000000000000000000000000000000000000000000000000000000050000005000000000000000001EFE9F
:3CA44C000000000000000000000000000000000000000000000000000000200000000000000000000000400000000000000000100000001000000000080080FECE
:3CA488000000000000000000000000000000000000000000000000000000000000000000000000002000000000000000000008000000000000000000000034FE3E
:3CA4C400000000000000000000000000000000000000000000000000000000000000000000000000000000000000000000000000000000000000000000001EFE40
:3CA50000000000000000000000000000000000000000000000000000000000000000000000000000000000000000000400000000000000010000000000000AFE12
:3CA53C000000000000000000000000000000000000000000000000000000000000000000000000000000000000000081000000000000008001000000000117FFCA
:3CA57800000000000000000000000000000000000000000000000000000000000000000000000000000000000000000000000000000000000000000000001EFE8B
:3CA5B4000000000000000000000000000000000000000000000000000000000000000000000000000000000000000000000000000000008002000000000094FE57
:3CA5F00002000000000000000000000000000000000000000000000000000000000000000000000000000000000000C000000000000000804A00000000200FFF75
:3CA62C0002000000000000000000000000000000000000000000000000000000000000000000000000000000000000240600000000000080040000002000E3FF40
:3CA66800000000000000000000000000000000000000000000000000000000000000000000000000000000000000000000000000000000000200000000000DFFA8
:3CA6A40002000000000000000000000000000000000000000000000000000000000000000000000000000000000000800600000000000000020000000000CBFF26
:3CA6E000020000000000000000000000000000000000000000000000000000000000000000000000000000000000000000000000000000004C000000004036FE7C
:3CA71C000000000000000000000000000000000000000000000000000000000000000000000000000000000000000000000000000000008001000082060062FF97
:3CA75800000000000000000000000000000000000000000000000000000000000000000000000000000000000000000000000000000000000000000000001EFEA9
:3CA794000000000000000000000000000000000000000000000000000000000000000000000000000000000000000000000000000000008002000080060072FE11
:3CA7D000020000000000000000000000000000000000000000000000000000000000000000000000000000000000000000000000000000802A0000C02800C7FFF3
:3CA80C00020000000000000000000000000000000000000000000000000000000000000000000000000000000000000000000000000000800400008800002BFFD8
:3CA84800000000000000000000000000000000000000000000000000000000000000000000000000000000000000000000000000000000000200000000001CFEB8
:3CA8840002000000000000000000000000000000000000000000000000000000000000000000000000000000000000000000000000000000020000800600CBFF44
:3CA8C000020000000000000000000000000000000000000000000000000000000000000000000000000000000000000000000000000000002C000020060045FFC4
:3CA8FC0000000000000000000000000000000000000000000000000000000000000000000000000000000000000000800C00000000000080090000A4160010FE43
:3CA93800000000000000000000000000000000000000000000000000000000000000000000000000000000000000000004000000000000000000000006003CFE9F
:3CA9740000000000000000000000000000000000000000000000000000000000000000000000000000000000000000800200000000000080020000800000B6FE6F
:3CA9B00002000000000000000000000000000000000000000000000000000000000000000000000000000000000000802200000000000080220000808600CBFF55
:3CA9EC0002000000000000000000000000000000000000000000000000000000000000000000000000000000000000800C000000000000800C000082000065FF2F
:3CAA2800000000000000000000000000000000000000000000000000000000000000000000000000000000000000000002000000000000000200000000003EFEB2
:3CAA6400020000000000000000000000000000000000000000000000000000000000000000000000000000000000000002000000000000000200008000008FFFA2
:3CAAA000020000000000000000000000000000000000000000000000000000000000000000000000000000000000000024000000000000002400004006006BFF80
:3CAADC000000000000000000000000000000000000000000000000000000000000000000000000000000000000000080120000801500008011000082160189FF65
:3CAB1800000000000000000000000000000000000000000000000000000000000000000000000000000000000000000002000000040000000000000000007CFE81
:3CAB540000000000000000000000000000000000000000000000000000000000000000000000000000000000000000800200008002000080020000800600F8FEC3
:3CAB900002000000000000000000000000000000000000000000000000000000000000000000000000000000000000802200008022000080220000C02020CFFFD3
:3CABCC0002000000000000000000000000000000000000000000000000000000000000000000000000000000000000801200008014000080140000A12040BFFED3
:3CAC08000000000000000000000000000000000000000000000000000000000000000000000000000000000000000000040000000200000002000000000069FFA0
:3CAC440002000000000000000000000000000000000000000000000000000000000000000000000000000000000000000200000002000000020000800600C9FF7E
:3CAC80000200000000000000000000000000000000000000000000000000000000000000000000000000000000000000240000002400000024000000060058FECE
:3CACBC00020000000000000000000000000000000000000000000000000000000000000000000000000000000000008100000080010000800100008202008EFEC7
:3CACF800000000000000000000000000000000000000000000000000000000000000000000000000000000000000000000000000000000000000000002003CFEE4
:3CAD3400000000000000000000000000000000000000000000000000000000000000000000000000000000000000000000000080020000800200008002001EFE41
:3CAD700000000000000000000000000000000000000000000000000000000000000000000000000000000000000000C00000008032000080320000C032008FFF03
:3CADAC0002000000000000000000000000000000000000000000000000000000000000000000000000000000000000240000008004000080040000800800C7FFEF
:3CADE800020000000000000000000000000000000000000000000000000000000000000000000000000000000000000006000000020000000200000000007AFEAB
:3CAE2400000000000000000000000000000000000000000000000000000000000000000000000000000000000000008000000000020000000200008006004BFF9E
:3CAE60000000000000000000000000000000000000000000000000000000000000000000000000000000000000000000060000003400000034000000860051FE73
:3CAE9C000200000000000000000000000000000000000000000000000000000000000000000000000000000000000000000000801100008001000090060149FF87
:3CAED8000000000000000000000000000000000000000000000000000000000000000000000000000000000000000000000000000000000000000000060078FEC2
:3CAF1400000000000000000000000000000000000000000000000000000000000000000000000000000000000000000000000080020000800200008000003CFE43
:3CAF5000000000000000000000000000000000000000000000000000000000000000000000000000000000000000000000000080020400808A0000A05620D1FE50
:3CAF8C000200000000000000000000000000000000000000000000000000000000000000000000000000000000000000000000801400008004000082202049FE66
:3CAFC800020000000000000000000000000000000000000000000000000000000000000000000000000000000000000000000000020000000200000000000DFF3B
:3CB0040000000000000000000000000000000000000000000000000000000000000000000000000000000000000000000000000002000000020000800000ADFFE0
:3CB04000000000000000000000000000000000000000000000000000000000000000000000000000000000000000000000000000040400008C0000400600F0FE0C
:3CB07C00020000000000000000000000000000000000000000000000000000000000000000000000000000000000000000000080010000800100008212010FFFF1
:3CB0B800000000000000000000000000000000000000000000000000000000000000000000000000000000000000000000000000000000000000000002003CFE20
:3CB0F400000000000000000000000000000000000000000000000000000000000000000000000000000000000000000000000080020000800200008002001EFE7E
:3CB13000000000000000000000000000000000000000000000000000000000000000000000000000000000000000000000000080120400800A0400C0023025FFA9
:3CB16C0002000000000000000000000000000000000000000000000000000000000000000000000000000000000000000000008004000080040000800810E3FE24
:3CB1A800020000000000000000000000000000000000000000000000000000000000000000000000000000000000000000000000020000000200000000000DFF59
:3CB1E40000000000000000000000000000000000000000000000000000000000000000000000000000000000000000000000000002000000020000800600CBFFDB
:3CB22000000000000000000000000000000000000000000000000000000000000000000000000000000000000000000000000000140400000C040000062146FF5E
:3CB25C0000000000000000000000000000000000000000000000000000000000000000000000000000000000000000000000008009000080110000D00601B9FE0E
:3CB2980000000000000000000000000000000000000000000000000000000000000000000000000000000000000000000080000000000000000000000600F0FE06
:3CB2D400000000000000000000000000000000000000000000000000000000000000000000000000000000000000000000000080020000800200008000003CFE80
:3CB3100002000000000000000000000000000000000000000000000000000000000000000000000000000000000000000000008002040080020200808E20EFFFD9
:3CB34C000200000000000000000000000000000000000000000000000000000000000000000000000000000000000000000000800C000080140000820030DBFE18
:3CB38800000000000000000000000000000000000000000000000000000000000000000000000000000000000000000000000000020000000200000000002DFF59
:3CB3C400020000000000000000000000000000000000000000000000000000000000000000000000000000000000000000000000020000000200008000008DFF3B
:3CB4000002000000000000000000000000000000000000000000000000000000000000000000000000000000000000000080000004040000040200400600F2FE4A
:3CB43C0002000000000000000000000000000000000000000000000080C0060000000000000000000000000000000081060000800900008011000082020157FF10
:3CB47800000000000000000000000000000000000000000000000000000006000000000000000000000000000000000000000000000000000000000002005AFE38
:3CB4B400000000000000000000000000000000000000000000000000000006000000000000000000000000000000000006000080020000800600008002001AFEAE
:3CB4F00000000000000000000000000000000000000000000000000000800600000000000000000000000000000000C00000008002020080060100C00A30C5FF11
:3CB52C000200000000000000000000000000000000000000000000000000000000000000000000000000000000000024000000800C00008006000080005089FE54
:3CB568000200000000000000000000000000000000000000000000000000000000000000000000000000000000000000000000000200000006000000000009FF95
:3CB5A40000000000000000000000000000000000000000000000000000800000000000000000000000000000000000800000000002000000000000800600C9FF1B
:3CB5E00000000000000000000000000000000000000000000000000000000000000000000000000000000000000000000000000004020000000000000E04F2FE27
:3CB61C0000000000000000000000000000000000000000000000000000000000000000000000000000000000000000000000000000000000000000881601E1FE74
:3CB658000000000000000000000000000000000000000000000000000000000000000000000000000000000000000000000000000000000000000000060078FE3A
:3CB69400000000000000000000000000000000000000000000000000000000000000000000000000000000000000000000000000000000000000008000009EFE5E
:3CB6D00002000000000000000000000000000000000000000000000000000000000000000000000000000000000000000000000010020000100200C00622BBFE77
:3CB70C00020000000000000000000000000000000000000000000000000000000000000000000000000000000000002200000001000000010000008200109FFFAB
:3CB748000080008000800080008000800080008000800080008000800080008000800080008000800080008000800080008000800080000000800080000007FF3F
:3CB78400020000000000000000000000000000000000000000000000000000000000000000000000000000000000000000000000000000000000000000002FFF59
:3CB7C000020000000000000000000000000000000000000000000000000000000000000000000000000000000000000000000040000000400000004006401CFE2B
:3CB7FC00000000000000000000000000000000000000000000000000000000000000000000000000000000000000004201000002010000020100000000005EFE6C
:3CB83800000000000000000000000000000000000000000000000000000000000000000000000000000000000000002000000008080100080801002000008EFEE6
:3CB87400000000000000000000000000000000000000000000000000000000000000000000000000000000000000000000000000000000000000000000001EFE7C
:3CB8B000000000000000000000000000000000000000000000000000000000000000000000000000000000000000000000000000000000000000000000001EFE40
:3CB8EC000000000000000000000000000000000000000000000000000000000000000000000000000000000000000000040000000000000000000008000052FEC4
:3CB928000000000000000000000000000000000000000000000000000000000000000000000000000000000000000020020000000000000002000000080096FE23
:3CB96400000000000000000000000000000000000000000000000000000000000000000000000000000000000000000000000000000000000000000000001EFE8B
:3CB9A000000000000000000000000000000000000000000000000000000000000000000000000000000000000000000000000000000000000000000000001EFE4F
:3CB9DC00000000000000000000000000000000000000000000000000000000000000000000000000000000000000000000000000000000000000000000001EFE13
:3CBA18000000000000000000000000000000000000000000000000000000000000000000000000000000000000000000000000800000000000000000000016FE5E
:3CBA5400000000000000000000000000000000000000000000000000000000000000000000000000000000000000000000000000000000000400000000010AFEA9
:3CBA9000000000000000000000000000000000000000000000000000000000000000000000000000000000000000000000000000000000004000000004001AFE1E
:3CBACC00000000000000000000000000000000000000000000000000000000000000000000000000000000000000000000000000000000000000000000001EFE22
:3CBB0800020000000000000000000000000000000000000000000000200000000000000000000000000000000000000000000000000000000000000000001CFEC5
:3CBB4400000000000000000000000000000000000000000000000000000000000000000000000000000000000000000000000000012000004100000040007AFFAA
:3CBB80000000000000000000000000000000000000000000000000000000000000000000000000000000000000000000000000800040000000000000000056FE75
:3CBBBC00000000000000000000000000000000000000000000000000000000000000000000000000000000000000000000000000000000000000000000001EFE31
:3CBBF800000000000000000000000000000000000000000000000000000000000000000000000000000000000000000000000000000000000000000000001EFEF5
:3CBC3400000000000000000000000000000000000000000000000000000000000000000000000000000000000000400010000000000000000000000000004AFF3B
:3CBC70000000000000000000000000000000000000000000000000000000000000000000000000000000000000000000800020000000200040000000100064FF25
:3CBCAC00000000000000000000000000000000000000000000000000000000000000000000000000000000000000000000000000000000000000000000001EFE40
:3CBCE800000000000000000000000000000000000000000000000000000000000000000000000000000000000000000400001000000000000000000000000AFE04
:3CBD2400000000000000000000000000000000000000000000000000000000000000000000000000000000000000000000000000000000000000000000001EFEC7
:3CBD6000000000000000000000000000000000000000000000000000000000000000000000000000000000000000000000000000000000000000000000001EFE8B
:3CBD9C000000000000000000000000000000000000000000000000000000000000000000000000000000000000000000000000800000000000000000000016FED7
:3CBDD8000000000000000000000000000000000000000000000000000000000000000000000000000000000000000000000000000000000008040000000412FE0F
:3CBE1400000000000000000000000000000000000000000000000000000000000000000000000000000000000000000000000000000000000000000000001EFED6
:3CBE5000000000000000000000000000000000000000000000000000000000000000000000000000000000000000000000000040001000000000000000000AFE5E
:3CBE8C00000000000000000000000000000000000000000000000000001000000000000000000000000000000000000000000000000000000001000100010EFE5B
:3CBEC800000000000000000000000000000000000000000000000000000000000000000000000000000000000000001000000000000200000002000000002EFEFE
:3CBF0400000000000000000000000000000000000000000000000000000000000000000000000000000000000000000000000000000000000000000000001EFEE5
:3CBF40000000000000000000000000000000000000000000000000000000000000000000000000000000000000000000000000100004001000010000200008FF79
:3CBF7C0000000000000000000000000000000000000000000000000000000000000000000000000000000000000000000000000000000000201000000008AEFFA4
:3CBFB800000000000000000000000000000000000000000000000000000000000000000000000000000000000000000000000000000000000800800000009EFE29
:3CBFF4000000000000000000000000000000000000000000000000000008000000000000000000000000000000000000000000280600000000000040080034FE61
:3CC03000000000000000000000000000000000000000000000000000000000000000000000000000000000000000000002000000000000000001002000001CFF96
:3CC06C00000000000000000000000000000000000000000000000000000000000000000000000000000000000000000000000000000000000001000100000EFE8A
:3CC0A800000000000000000000000000000000000000000000000000000000000000000000000000000000000000000000000000000000000000000000001EFE40
:3CC0E40000000400040004800000008000800480040000000480040000000000000000000000048004800000048004000480040000000000008000800000D6FE98
:3CC120000000008000800000048004000400000000800480000000800480048004800480048000000000048000000080000000800480048004A004A000007CFEF1
:3CC15C000000048004800480048004800480048004800480048004800480048004800480048004800480048004800480048004800480048084C00488000092FE63
:3CC1980000000400040004800000008000800480040000000480040000000000000000000000048004800000048004000480040000000000008000800000D6FEE3
:3CC1D400000000800080000004800400040000000080048000000080048004800480048004800000000004800000008000000080048004800480048000005EFE9B
:3CC210000000008000800000048004000400000000800480000000800480048004800480048000000000048000000080000000800480048004000440000096FEE6
:02C24C00FFFFF2
:00000001FF
